:0200000480007A
:10000000B72F0000938F0F8073900F306F00400365
:100010001300000013000000130000001300000094
:100020001300000013000000130000001300000084
:100030001300000013000000130000001300000074
:100040009702000093824211739052309300000097
:10005000130100009301000013020000930200004E
:100060001303000093030000130400009304000036
:10007000130500009305000013060000930600001E
:100080001307000093070000130800009308000006
:100090001309000093090000130A0000930A0000EE
:1000A000130B0000930B0000130C0000930C0000D6
:1000B000130D0000930D0000130E0000930E0000BE
:1000C000130F0000930F000097110200938141BFAE
:1000D0001705020013050543979503009385C56E28
:1000E00013060000EF00001A170502001305853CF7
:1000F000970502009385853C13060000EF008018E9
:1001000017A503001305856C97B503009385C56B90
:1001100037B6ABAB1306B6BAEF00C01617B1030083
:100120001301C16AEF7040399392120093D212000A
:100130009382D2FF638A02008322010013014100EF
:100140006F0000177300203083220100130141006B
:10015000730020301301C1FF23205100F32220340B
:10016000E3C402FC8322010013014100130141F8A2
:1001700023221100232421002326310023284100BB
:10018000232A5100232C6100232E71002320810299
:10019000232291022324A1022326B1022328C10293
:1001A000232AD102232CE102232EF1022320010570
:1001B0002322110523242105232631052328410567
:1001C000232A5105232C6105232E71052320810745
:1001D000232291072324A1072326B1072328C1073F
:1001E000232AD107232CE107232EF107732520347E
:1001F000F3251034130601006F000000731015344E
:1002000083204100032181008321C10003220101D9
:1002100083224101032381018323C10103240102BD
:1002200083244102032581028325C10203260103A1
:1002300083264103032781038327C1030328010485
:1002400083284104032981048329C104032A010569
:10025000832A4105032B8105832BC105032C01064D
:10026000832C4106032D8106832DC106032E010731
:10027000832E4107032F8107832FC1071301C10775
:10028000730020302320C5006376B50013054500B8
:100290006FF05FFF678000000000000000000000BA
:1002A000000000000000000000000000000000004E
:1002B000130101F8232011002322210023243100FF
:1002C0002326410023285100232A6100232C71009A
:1002D000232E8100232091022322A1022324B10294
:1002E0002326C1022328D102232AE102232CF10272
:1002F000232E010323201105232221052324310568
:100300002326410523285105232A6105232C710545
:10031000232E8105232091072322A1072324B1073F
:100320002326C1072328D107232AE107232CF1071D
:100330009702020083A2021823A02200F3221034A5
:10034000232E5106EF00804617010200032181167B
:10035000032101008322C10773901234B7220000E9
:100360009382028873A00230832001000322C1001F
:100370008322010103234101832381010324C1015D
:100380008324010203254102832581020326C10241
:100390008326010303274103832781030328C10325
:1003A000832801040329410483298104032AC10409
:1003B000832A0105032B4105832B8105032CC105ED
:1003C000832C0106032D4106832D8106032EC106D1
:1003D000832E0107032F4107832F81071301010893
:1003E00073002030970202009382C21123A01200F2
:1003F00023A2220023A4320023A6420023A85200F5
:1004000023AA620023AC720023AE820023A09202D2
:1004100023A2A20223A4B20223A6C20223A8D202CC
:1004200023AAE20223ACF20223AE020323A01205A8
:1004300023A2220523A4320523A6420523A85205A0
:1004400023AA620523AC720523AE820523A092077E
:1004500023A2A20723A4B20723A6C20723A8D20778
:1004600023AAE20723ACF207EF6010731701020022
:1004700003214104032101008322C1077390123438
:10048000B72200009382028873A00230832001000B
:100490000322C1008322010103234101832381013F
:1004A0000324C10183240102032541028325810223
:1004B0000326C10283260103032741038327810307
:1004C0000328C103832801040329410483298104EB
:1004D000032AC104832A0105032B4105832B8105CF
:1004E000032CC105832C0106032D4106832D8106B3
:1004F000032EC106832E0107032F4107832F810797
:10050000130101087300203097020200938282FFDA
:1005100083A0020003A1420083A1820003A2C200C3
:1005200083A2020103A3420183A3820103A4C201A7
:1005300083A4020203A5420283A5820203A6C2028B
:1005400083A6020303A7420383A7820303A8C2036F
:1005500083A8020403A9420483A9820403AAC20453
:1005600083AA020503AB420583AB820503ACC20537
:1005700083AC020603AD420683AD820603AEC2061B
:1005800083AE020703AFC20983AF82076780000012
:1005900073700430130101F823201100232221007D
:1005A000232431002326410023285100232A6100FF
:1005B000232C7100232E8100232091022322A102EB
:1005C0002324B1022326C1022328D102232AE102D7
:1005D000232CF102232E01032320110523222105C0
:1005E000232431052326410523285105232A6105AB
:1005F000232C7105232E8105232091072322A10797
:100600002324B1072326C1072328D107232AE10782
:10061000232CF1079702020083A2C2E923A0220043
:10062000232E1106EF20D05817010200032181E884
:10063000032101008322C10773901234B722000006
:100640009382028873A00230832001000322C1003C
:100650008322010103234101832381010324C1017A
:100660008324010203254102832581020326C1025E
:100670008326010303274103832781030328C10342
:10068000832801040329410483298104032AC10426
:10069000832A0105032B4105832B8105032CC1050A
:1006A000832C0106032D4106832D8106032EC106EE
:1006B000832E0107032F4107832F810713010108B0
:1006C0007300203097070200938787DF03A7070096
:1006D0009307F0FF6306F700737004306F000000AB
:1006E000737004306F000000130101FF2326A10086
:1006F0008327C100739047301300000013010101EC
:1007000067800000130101FFF32740302326F1002A
:1007100073F043308327C1001385070013010101E3
:1007200067800000130101FF2326A1002324B100EC
:100730002322C1008327C1009387C7FF2326F1002E
:10074000032781008327C10023A0E7008327C1007E
:10075000938787FA2326F100032741008327C100EE
:1007600023A0E7008327C100938787FE2326F1009B
:1007700093870100138707008327C10023A0E700A8
:100780008327C100938747FF2326F1001707000046
:10079000130787F38327C10023A0E7008327C10045
:1007A000138507001301010167800000130101FF99
:1007B00023261100EF60D033EF20101693070500B9
:1007C00063840700EF20D03E130000008320C100A7
:1007D0001301010167800000130101FF2326A1001E
:1007E0008327C100138787008327C10023A2E70066
:1007F0008327C1001307F0FF23A4E7008327C1006C
:10080000138787008327C10023A6E7008327C10041
:10081000138787008327C10023A8E7008327C1002F
:1008200023A00700130000001301010167800000EE
:10083000130101FF2326A1008327C10023A807007D
:10084000130000001301010167800000130101FE85
:100850002326A1002324B1008327C10083A74700DA
:10086000232EF100832781000327C10123A2E70083
:100870008327C10103A787008327810023A4E70002
:100880008327C10183A787000327810023A2E700F4
:100890008327C1010327810023A4E7008327810068
:1008A0000327C10023A8E7008327C10083A707000F
:1008B000138717008327C10023A0E700130000005F
:1008C0001301010267800000130101FE2326A1002D
:1008D0002324B1008327810083A70700232CF10084
:1008E000032781019307F0FF631AF7008327C100F4
:1008F00083A70701232EF1006F0040038327C10067
:1009000093878700232EF1006F0000018327C10128
:1009100083A74700232EF1008327C10183A7470047
:1009200083A7070003278101E372F7FE8327C10134
:1009300003A747008327810023A2E70083278100C4
:1009400083A747000327810023A4E70083278100B2
:100950000327C10123A4E7008327C10103278100E6
:1009600023A2E700832781000327C10023A8E70013
:100970008327C10083A70700138717008327C100BF
:1009800023A0E700130000001301010267800000AC
:10099000130101FE2326A1008327C10083A70701BD
:1009A000232EF1008327C10083A747000327C1003E
:1009B0000327870023A4E7008327C10083A78700BC
:1009C0000327C1000327470023A2E7008327C101B3
:1009D00083A747000327C100631AF7008327C100DC
:1009E00003A787008327C10123A2E7008327C10053
:1009F00023A807008327C10183A707001387F7FFF8
:100A00008327C10123A0E7008327C10183A7070033
:100A1000138507001301010267800000130101FD27
:100A200023261102232481022326A1002324B100BE
:100A30008327C100232EF1008327C101639607009D
:100A4000737004306F000000EF3010418327C10144
:100A500003A407008327C10103A7C7038327C1019C
:100A600083A707049385070013050700EFA08030D4
:100A7000930705003307F4008327C10123A2E70091
:100A80008327C10123AC07028327C10103A7070005
:100A90008327C10123A4E7008327C10103A4070022
:100AA0008327C10183A7C7031387F7FF8327C101EA
:100AB00083A707049385070013050700EFA0802B89
:100AC000930705003307F4008327C10123A6E7003D
:100AD0008327C1011307F0FF23A2E7048327C10185
:100AE0001307F0FF23A4E70483278100639A07021A
:100AF0008327C10183A70701638407048327C101FA
:100B00009387070113850700EF20504C130705005A
:100B1000930710006316F702EFF09FA76F004002E3
:100B20008327C1019387070113850700EFF0DFCA10
:100B30008327C1019387470213850700EFF0DFC9C0
:100B4000EF30903593071000138507008320C10212
:100B5000032481021301010367800000130101FDDA
:100B6000232611022326A1002324B10093070600A7
:100B7000A303F100232C01008327C1006396070023
:100B8000737004306F0000008327810063960700B4
:100B9000232E01006F00C001832581000325C100C1
:100BA000EFA0401D9307050093871700232EF10047
:100BB0008327C1019387470513850700EF50006E17
:100BC000232AA1008327410163820706832781002E
:100BD000639A0700832741010327410123A0E7000F
:100BE0006F00400183274101138747058327410197
:100BF00023A0E700832741010327C10023AEE702BA
:100C0000832741010327810023A0E70493051000F7
:100C100003254101EFF09FE0832741010347710065
:100C20002388E70483274101232CF10083278101D6
:100C300063960700737004306F0000008327810102
:100C4000138507008320C1021301010367800000A0
:100C5000130101FD2326110293070500A307F100EC
:100C600013054005EF508063232EA1008327C101A7
:100C7000638C07088327C10123A207008327C101D2
:100C800023A007008327C10123A407008327C101F4
:100C900023A607008327C10123AC07028327C101D4
:100CA0001307100023AEE7028327C10123A0070426
:100CB0008327C1011307F0FF23A2E7048327C101A3
:100CC0001307F0FF23A4E7048327C1010347F100C2
:100CD0002388E7048327C101938707011385070051
:100CE000EFF09FAF8327C101938747021385070069
:100CF000EFF09FAE9306000013060000930500007E
:100D00000325C101EF00001E8327C10113850700E1
:100D10008320C1021301010367800000130101FD5C
:100D200023261102232481022326A1008327C10048
:100D3000232CF10083278101639607007370043030
:100D40006F0000008327810103A44700EF3000609B
:100D5000930705006312F4048327810183A7C7006A
:100D60001387F7FF8327810123A6E70083278101EB
:100D700083A7C700639C07009306000013060000CA
:100D80009305000003258101EF00C01593071000B3
:100D9000232EF1006F008000232E01008327C10164
:100DA000138507008320C10203248102130101037C
:100DB00067800000130101FD232611022324810214
:100DC0002326A1002324B1008327C100232CF10096
:100DD0008327810163960700737004306F00000061
:100DE0008327810103A44700EF3040569307050095
:100DF0006312F4028327810183A7C70013871700BA
:100E00008327810123A6E70093071000232EF1001A
:100E10006F00C003930600000326810093050000C5
:100E200003258101EF00C058232EA1000327C10133
:100E300093071000631CF7008327810183A7C70075
:100E4000138717008327810123A6E7008327C101A9
:100E5000138507008320C1020324810213010103CB
:100E600067800000130101FD232611022326A10043
:100E70002324B1008327C1006396070073700430F8
:100E80006F000000032781008327C10063F6E7009D
:100E9000737004306F0000001306200093050000FB
:100EA0000325C100EFF09FCB232EA1008327C101B2
:100EB000638807008327C1010327810023ACE70271
:100EC0008327C10163960700737004306F00000030
:100ED0008327C101138507008320C1021301010389
:100EE00067800000130101FC232E11022326A100BC
:100EF0002324B1002322C1002320D1002326010294
:100F00008327C1002324F10283278102639607000F
:100F1000737004306F00000083278100639807001E
:100F20008327810283A707046396070093071000B5
:100F30006F00800093070000639607007370043011
:100F40006F0000000327010093072000631AF700D9
:100F50008327810203A7C703930710006316F700D6
:100F6000930710006F00800093070000639607004E
:100F7000737004306F000000EF30803F930705006E
:100F800063960700832741006396070093071000CC
:100F90006F008000930700006396070073700430B1
:100FA0006F000000EF30406B8327810203A78703A7
:100FB0008327810283A7C7036368F7000327010023
:100FC000930720006310F7060326010083258100A4
:100FD00003258102EF00101C2322A1028327810236
:100FE00083A747026384070283278102938747020E
:100FF00013850700EF20807D13070500930710007D
:10100000631CF700EFF0CFD86F0000018327410287
:1010100063840700EFF0CFD7EF300068930710002C
:101020006F00400F8327410063980700EF30C066D0
:10103000930700006F00000E8327C102639C070026
:101040009307C10113850700EF20501D930710007F
:101050002326F102EF304064EF10D049EF30C05F3B
:101060008327810203A747049307F0FF6316F70065
:101070008327810223A207048327810203A7870411
:101080009307F0FF6316F7008327810223A4070468
:10109000EF308060130741009307C10193050700FB
:1010A00013850700EF20501C93070500639C07047D
:1010B00003258102EF00504693070500638C070269
:1010C00083278102938707010327410093050700C7
:1010D00013850700EF20004A03258102EF00902CC2
:1010E000EF10904393070500E39E07EAEFF04FCA25
:1010F0006FF05FEB03258102EF00D02AEF10D041A3
:101100006FF05FEA03258102EF00D029EF10D04095
:1011100093070000138507008320C1031301010416
:1011200067800000130101FD232611022326A10080
:101130002324B1002322C1002320D1008327C10032
:10114000232CF1008327810163960700737004301C
:101150006F000000832781006398070083278101C7
:1011600083A7070463960700930710006F008000B1
:101170009307000063960700737004306F0000004F
:101180000327010093072000631AF70083278101DA
:1011900003A7C703930710006316F7009307100017
:1011A0006F0080009307000063960700737004309F
:1011B0006F000000EFF00FD593070500232AF10020
:1011C0008327810103A787038327810183A7C7039F
:1011D0006368F70003270100930720006310F708F6
:1011E000032601008325810003258101EF00807A19
:1011F0008327810103A787049307F0FF6310F70497
:101200008327810183A74702638407048327810121
:101210009387470213850700EF20405B9307050083
:101220006388070283274100638407028327410004
:101230001307100023A0E7006F00800183278101BE
:1012400083A78704138717008327810123A4E7045A
:1012500093071000232EF1006F008000232E010061
:101260008327410113850700EFF00FC88327C101D1
:10127000138507008320C10213010103678000006A
:10128000130101FD232611022326A1002324B1000E
:101290008327C100232CF100832781016396070077
:1012A000737004306F0000008327810183A7070457
:1012B00063860700737004306F000000832781018C
:1012C00083A70700639807008327810183A747004E
:1012D00063960700930710006F00800093070000DB
:1012E00063960700737004306F000000EFF08FC149
:1012F00093070500232AF1008327810103A78703B1
:101300008327810183A7C7036372F70883278101BD
:1013100083A78703138717008327810123ACE70284
:101320008327810103A787049307F0FF6310F70465
:101330008327810183A747026384070483278101F0
:101340009387470213850700EF2040489307050065
:101350006388070283278100638407028327810053
:101360001307100023A0E7006F008001832781018D
:1013700083A78704138717008327810123A4E70429
:1013800093071000232EF1006F008000232E010030
:101390008327410113850700EFF00FB58327C101B3
:1013A000138507008320C102130101036780000039
:1013B000130101FC232E11022326A1002324B100D6
:1013C0002322C1002320D100232601028327C1004C
:1013D0002324F1028327810263960700737004308F
:1013E0006F00000083278100639807008327810234
:1013F00083A7070463960700930710006F0080001F
:101400009307000063960700737004306F000000BC
:10141000EF201076930705006396070083274100AD
:1014200063960700930710006F0080009307000089
:1014300063960700737004306F000000EF30C02126
:101440008327810283A787036382070C8327810296
:1014500083A7C7002322F10283258100032581028F
:10146000EF00806B832701006392070683278102C8
:1014700083A787031387F7FF8327810223ACE70243
:101480008327810283A70700639A0700EF30802B30
:10149000130705008327810223A2E7008327810227
:1014A00083A70701638E07048327810293870701BF
:1014B00013850700EF208031130705009307100004
:1014C0006310F704EFF0CF8C6F0080038327810255
:1014D0000327410223A6E7008327810283A747024F
:1014E00063800702832781029387470213850700E1
:1014F000EF20C02D9307050063840700EFF04F89AC
:10150000EF308019930710006F008011832741008E
:1015100063980700EF304018930700006F004010F9
:101520008327C102639C07009307C101138507004D
:10153000EF20C04E930710002326F102EF30C015B4
:10154000EF10407BEF3040118327810203A747044F
:101550009307F0FF6316F7008327810223A2070495
:101560008327810203A787049307F0FF6316F70020
:101570008327810223A40704EF30001213074100E0
:101580009307C1019305070013850700EF20C04DA5
:1015900093070500639E070603258102EF00406F55
:1015A00093070500638E07048327810283A7070042
:1015B000639E0700EF30400A8327810283A747001C
:1015C00013850700EF20D05FEF30000D83278102E5
:1015D00093874702032741009305070013850700FF
:1015E000EF10507903258102EF00C05BEF10C0724D
:1015F00093070500E39407E4EFE09FF96FF01FE421
:1016000003258102EF00005AEF1000716FF01FE315
:1016100003258102EF000059EF10007093070000CE
:10162000138507008320C1031301010467800000B4
:10163000130101FD232611022326A1002324B1005A
:101640002322C1008327C100232CF10083278101BD
:1016500063960700737004306F00000083278100D9
:10166000639807008327810183A707046396070017
:10167000930710006F008000930700006396070037
:10168000737004306F000000EFF0CF879307050000
:10169000232AF1008327810183A787036388070832
:1016A0008325810003258101EF0000478327810105
:1016B00083A787031387F7FF8327810123ACE70202
:1016C0008327810103A747049307F0FF6310F70402
:1016D0008327810183A7070163840704832781018E
:1016E0009387070113850700EF20400E930705003D
:1016F0006388070283274100638407028327410030
:101700001307100023A0E7006F00800183278101E9
:1017100083A74704138717008327810123A2E704C7
:1017200093071000232EF1006F008000232E01008C
:101730008327410113850700EFE01FFB8327C101C9
:10174000138507008320C102130101036780000095
:10175000130101FD232611022326A1002324B10039
:101760008327C100232CF1008327810163960700A2
:10177000737004306F0000008327810063980700B6
:101780008327810183A7070463960700930710004E
:101790006F008000930700006396070073700430A9
:1017A0006F0000008327810183A707046396070069
:1017B000737004306F000000EFE0DFF49307050062
:1017C000232AF1008327810183A78703638A070205
:1017D0008327810183A7C7002328F1008325810087
:1017E00003258101EF004033832781010327010195
:1017F00023A6E70093071000232EF1006F0080005E
:10180000232E01008327410113850700EFE0DFED60
:101810008327C101138507008320C102130101033F
:1018200067800000130101FD232611022326A10079
:101830008327C10063960700737004306F000000B7
:10184000EF2090618327C10083A78703232EF10037
:10185000EF2090648327C101138507008320C10214
:101860001301010367800000130101FD232611020B
:101870002326A1008327C100232EF1008327C10165
:1018800063960700737004306F000000EF20D05C97
:101890008327C10103A7C7038327C10183A7870348
:1018A000B307F740232CF100EF20105F832781015D
:1018B000138507008320C102130101036780000024
:1018C000130101FE2326A1008327C10063960700B0
:1018D000737004306F0000008327C10083A7870363
:1018E000232EF1008327C101138507001301010294
:1018F00067800000130101FD232611022326A100A9
:101900008327C100232EF1008327C10163960700BE
:10191000737004306F0000000325C101EF004052D6
:101920000325C101EF405037130000008320C1029E
:101930001301010367800000130101FF2326A100AA
:101940008327C10083A7C704138507001301010182
:1019500067800000130101FF2326A1002324B100AA
:101960008327C1000327810023A6E704130000009A
:101970001301010167800000130101FF2326A1006C
:101980008327C10083C707051385070013010101E1
:1019900067800000130101FD232611022326A10008
:1019A0002324B1002322C100232E01008327C1007C
:1019B00083A70704639807028327C10083A7070052
:1019C000639807128327C10083A747001385070088
:1019D000EF20D034232EA1008327C10023A20700CB
:1019E0006F00001183274100639407068327C1001D
:1019F00003A787008327C10083A707041386070076
:101A00008325810013050700EF40D03F8327C100E5
:101A100003A787008327C10083A707043307F700C4
:101A20008327C10023A4E7008327C10003A7870001
:101A30008327C10083A74700636CF70A8327C1008F
:101A400003A707008327C10023A4E7006F00400A13
:101A50008327C10003A7C7008327C10083A707040A
:101A6000138607008325810013050700EF40903996
:101A70008327C10003A7C7008327C10083A70704EA
:101A8000B307F0403307F7008327C10023A6E70020
:101A90008327C10003A7C7008327C10083A70700CE
:101AA0006372F7028327C10003A747008327C100A1
:101AB00083A70704B307F0403307F7008327C1006B
:101AC00023A6E70003274100930720006312F702D3
:101AD0008327C10083A78703638C07008327C10086
:101AE00083A787031387F7FF8327C10023ACE7028F
:101AF0008327C10083A78703138717008327C100AB
:101B000023ACE7028327C101138507008320C102AC
:101B10001301010367800000130101FE232E110051
:101B20002326A1002324B1008327C10083A7070433
:101B3000638207068327C10003A7C7008327C1006C
:101B400083A707043307F7008327C10023A6E70014
:101B50008327C10003A7C7008327C10083A74700CD
:101B6000636AF7008327C10003A707008327C1002A
:101B700023A6E7008327C10003A7C7008327C1006E
:101B800083A7070413860700930507000325810038
:101B9000EF405027130000008320C1011301010210
:101BA00067800000130101FE232E11002326A100EF
:101BB000EF20902A6F0000048327C10083A747020B
:101BC000638207048327C1009387470213850700B8
:101BD000EF10D03F9307050063840700EF10D07823
:101BE0008327C10083A787041387F7FF8327C100DA
:101BF00023A4E7048327C10083A78704E34EF0FAF8
:101C00006F008000130000008327C1001307F0FF5E
:101C100023A4E704EF205028EF2010246F000004D5
:101C20008327C10083A70701638207048327C100BC
:101C30009387070113850700EF10503993070500BC
:101C400063840700EF1050728327C10083A7470405
:101C50001387F7FF8327C10023A2E7048327C1006E
:101C600083A74704E34EF0FA6F00800013000000E2
:101C70008327C1001307F0FF23A2E704EF20D02140
:101C8000130000008320C1011301010267800000DE
:101C9000130101FD232611022326A100EF20D01BF2
:101CA0008327C10083A78703639807009307100069
:101CB000232EF1006F008000232E0100EF20D01DA5
:101CC0008327C101138507008320C102130101038B
:101CD00067800000130101FE2326A1008327C100B5
:101CE00063960700737004306F0000008327C10003
:101CF00083A787036398070093071000232EF10042
:101D00006F008000232E01008327C1011385070087
:101D10001301010267800000130101FD2326110257
:101D20002326A100EF2050138327C10003A78703B8
:101D30008327C10083A7C7036318F7009307100028
:101D4000232EF1006F008000232E0100EF20D0141D
:101D50008327C101138507008320C10213010103FA
:101D600067800000130101FE2326A1008327C10024
:101D700063960700737004306F0000008327C10072
:101D800003A787038327C10083A7C7036318F7004E
:101D900093071000232EF1006F008000232E010016
:101DA0008327C1011385070013010102678000002A
:101DB000130101FE2326A1002324B100232E0100DC
:101DC0006F008006178703001307479C8327C10114
:101DD00093973700B307F70083A7070063900704C2
:101DE000178703001307879A8327C101939737004A
:101DF000B307F7000327810023A0E700178703003C
:101E00001307C7988327C10193973700B307F700DB
:101E10000327C10023A2E7006F00C0018327C1018F
:101E200093871700232EF1000327C1019307700049
:101E3000E3FAE7F8130000001301010267800000D5
:101E4000130101FE2326A100232E01006F00C00410
:101E500017870300130787938327C10193973700E0
:101E6000B307F70083A747000327C1006310F702F9
:101E700017870300130787918327C10193973700C2
:101E8000B307F70023A007006F00C0018327C1013B
:101E900093871700232EF1000327C10193077000D9
:101EA000E3F8E7FA13000000130101026780000065
:101EB000130101FD232611022326A1002324B100D2
:101EC0002322C1008327C100232EF100EF20C07818
:101ED0008327C10103A747049307F0FF6316F700A8
:101EE0008327C10123A207048327C10103A7870415
:101EF0009307F0FF6316F7008327C10123A40704AB
:101F0000EF2080798327C10183A78703639E0700A1
:101F10008327C1019387470203264100832581005F
:101F200013850700EF10007F0325C101EFF09FC765
:101F3000130000008320C102130101036780000029
:101F4000130101FC232E1102232EA100232CB1002A
:101F50002328D1002326E1002324F10023220101BC
:101F60002320110193070600231BF1008327C101E1
:101F700063960700737004306F0000000327C100F0
:101F80009307400063F6E700737004306F000000B1
:101F9000835761018325410013850700EF10D07E30
:101FA0002324A102832781026386071C83278102E1
:101FB00003A7070383566101B70700409387F7FF24
:101FC000B387F60093972700B307F7002322F102A7
:101FD0008327410293F7C7FF2322F102832741029F
:101FE00093F7370063860700737004306F000000BA
:101FF0008357610113870700832601000326C10070
:102000008325810103258102EF1050410326010140
:102010008325C10103254102EFE0CFF0130705003E
:102020008327810223A0E7008327810063880700BC
:10203000832781000327810223A0E700EF20C061EE
:1020400097E701009387076183A7070013871700AD
:1020500097E701009387076023A0E70097E7010057
:102060009387474583A707006398070297E7010016
:10207000938747440327810223A0E70097E70100E5
:102080009387475D03A70700930710006312F704C7
:10209000EF10904B6F00C00397E701009387475CF8
:1020A00083A707006396070297E70100938787409D
:1020B00083A7070083A7C7020327C100636AF7004D
:1020C00097E701009387073F0327810223A0E700DA
:1020D00097E701009387C75983A707001387170065
:1020E00097E701009387C75823A0E70097E701000F
:1020F0009387075803A707008327810223A4E704D7
:102100008327810203A7C70297E70100938707553A
:1021100083A7070063FCE7008327810203A7C702A8
:1021200097E701009387875323A0E7008327810265
:1021300003A7C7029307070093972700B387E70019
:102140009397270017E70100130787433387E700BA
:1021500083278102938747009385070013050700B3
:10216000EFE0CFEE930710002326F102EF20C052DC
:102170006F00C0009307F0FF2326F1020327C1027E
:10218000930710006318F70297E701009387474D04
:1021900083A707006380070297E7010093878731D1
:1021A00083A7070083A7C7020327C10063F4E700E2
:1021B000EFE00FBE8327C102138507008320C10310
:1021C0001301010467800000130101FD23261102A1
:1021D0002326A100EF2040488327C100639A07000F
:1021E00097E701009387072D83A707006F00800002
:1021F0008327C100232EF1008327C1019387470065
:1022000013850700EFE0CFF88327C10183A787027A
:10221000638A07008327C10193878701138507001D
:10222000EFE00FF78327C1019387470093850700ED
:1022300017E501001305453FEFE04FE197E7010087
:102240009387C73F83A707001387170097E701000D
:102250009387C73E23A0E70097E701009387474194
:1022600083A707001387170097E70100938747406C
:1022700023A0E700EF20404297E701009387473E05
:1022800083A707006382070497E7010093878722EB
:1022900083A707000327C1016312F70297E7010034
:1022A0009387873D83A70700638607007370043018
:1022B0006F000000EFE0CFAD6F000001EF20C039EC
:1022C000EF208001EF20403D130000008320C10279
:1022D0001301010367800000130101FD2326110291
:1022E0002326A1002324B100232E01008327C1004F
:1022F00063960700737004306F000000832781002D
:1023000063960700737004306F00000097E70100C8
:102310009387873683A707006386070073700430AE
:102320006F000000EF00101D97E701009387C73290
:1023300083A70700232CF1008327C10083A7070090
:1023400003278100B307F700232AF1008327C10088
:1023500083A70700032781016376F7028327C10063
:1023600083A70700032741016370F7040327410196
:102370008327810163FAE70293071000232EF100FF
:102380006F0080028327C10083A707000327410154
:102390006368F700032741018327810163F6E700A3
:1023A00093071000232EF1008327C100032741016A
:1023B00023A0E7008327C1016382070297E701009A
:1023C0009387470F83A7070093874700138507006C
:1023D000EFE00FDC03254101EF10502FEF00D01389
:1023E0002328A1008327010163940700EFE04F9A9F
:1023F000130000008320C102130101036780000065
:10240000130101FD232611022326A100232E010022
:102410008327C1006380070697E701009387C725DC
:1024200083A7070063860700737004306F00000005
:10243000EF00500C97E701009387072283A707005E
:102440000327C100B307F700232CF10097E7010031
:102450009387470683A707009387470013850700E4
:10246000EFE00FD303258101EF105026EF00D00AD3
:10247000232EA1008327C10163940700EFE04F9151
:10248000130000008320C1021301010367800000D4
:10249000130101FD232611022326A1008327C10079
:1024A000232CF100832781016396070073700430A9
:1024B0006F00000097E701009387C7FF83A707001D
:1024C000032781016316F700232E01006F00400AE5
:1024D000EF2080188327810183A74701232AF10079
:1024E000EF20801B97E701009387471283A707001F
:1024F00003274101630CF70097E701009387471119
:1025000083A70700032741016318F7009307200002
:10251000232EF1006F00C0050327410197E701005A
:10252000938707126314F7028327810183A7870229
:102530006398070093073000232EF1006F004003DB
:1025400093072000232EF1006F0080020327410132
:1025500097E701009387470D6318F7009307400042
:10256000232EF1006F00C00093071000232EF1000E
:102570008327C101138507008320C10213010103D2
:1025800067800000130101FD232611022326A1000C
:10259000EF20800C8327C100639A070097E70100B2
:1025A000938747F183A707006F0080008327C1004E
:1025B000232EF1008327C10183A7C702232CF1003A
:1025C000EF20800D83278101138507008320C1023E
:1025D0001301010367800000130101FD232611028E
:1025E0002326A100EFE00F9293070500232EF100B0
:1025F0008327C100639A070097E70100938787EB61
:1026000083A707006F0080008327C100232CF100FF
:102610008327810183A7C702232AF1008327C101F1
:1026200013850700EFE04F8C8327410113850700D6
:102630008320C1021301010367800000130101FD23
:10264000232611022326A1002324B100232E0100FA
:10265000032781009307400063F6E700737004309E
:102660006F000000032781009307400063F6E70036
:10267000930740002324F100EF10107E8327C10050
:10268000639A070097E701009387C7E283A70700D3
:102690006F0080008327C100232CF1008327810174
:1026A00083A70705232AF10003274101832781001F
:1026B000630EF716032781008327410163FEE702BB
:1026C00097E70100938707DF83A7070003278101AE
:1026D0006302F70497E701009387C7DD83A707002C
:1026E00083A7C702032781006366F70293071000E0
:1026F000232EF1006F00000297E70100938787DB2C
:1027000083A70700032781016316F70093071000D2
:10271000232EF1008327810183A7C7022328F1001C
:102720008327810103A707058327810183A7C702A8
:102730006318F700832781010327810023A6E7029E
:10274000832781010327810023A8E70483278101D0
:1027500083A7870163CC07001307500083278100FC
:102760003307F7408327810123ACE70083278101EA
:1027700083A64701032701019307070093972700CA
:10278000B387E7009397270017E70100130747DF98
:10279000B387E7006396F600930710006F00800090
:1027A00093070000638C0706832781019387470006
:1027B00013850700EFE0CF9D8327810103A7C702A0
:1027C00097E70100938787E983A7070063FCE70089
:1027D0008327810103A7C70297E70100938707E8D2
:1027E00023A0E7008327810103A7C70293070700FF
:1027F00093972700B387E7009397270017E7010017
:10280000130707D83387E7008327810193874700A1
:102810009385070013050700EFE04F830327C101ED
:10282000930710006314F700EFD09FD6EF10D06627
:10283000130000008320C102130101036780000020
:10284000130101FD232611022326A100EF10D06001
:102850008327C100639A070097E70100938787C524
:1028600083A707006F0080008327C100232EF1009B
:102870008327C1019387470013850700EFE04F913D
:102880008327C10183A78702638A07008327C101C9
:102890009387870113850700EFE08F8F8327C1019E
:1028A000938747009385070017E50100130545D975
:1028B000EFD0DFF9EF10505E97E70100938787BFF5
:1028C00083A707000327C1016314F70697E70100F8
:1028D000938707D983A707006382070297E7010060
:1028E000938787D983A70700638607007370043036
:1028F0006F000000EFD0DFC96F00400597E70100CF
:10290000938707D403A7070097E70100938787D42D
:1029100083A70700631AF70097E70100938787B939
:1029200023A007006F008002EF0090286F000002D4
:1029300097E701009387C7D283A707006388070042
:10294000EF109051EF105019EF10105513000000C8
:102950008320C1021301010367800000130101FEFF
:102960002326A100232E01008327C100232CF10080
:102970008327C10063960700737004306F00000066
:102980008327810103A7470197E70100938747CB7E
:102990006316F700930710006F0080009307000094
:1029A000638E07028327810103A7870297E701004F
:1029B000938747C66304F7028327810183A78702B1
:1029C00063960700930710006F00800093070000D4
:1029D0006386070093071000232EF1008327C101AF
:1029E000138507001301010267800000130101FD38
:1029F000232611022326A1008327C100232EF100E4
:102A00008327C10063960700737004306F000000D5
:102A10008327C1016384070C97E70100938787A987
:102A200083A707000327C101630AF70AEF10D0420A
:102A30000325C101EFF09FF2130705009307100073
:102A4000631CF7088327C10193874700138507009C
:102A5000EFD01FF48327C10103A7C70297E7010046
:102A60009387C7BF83A7070063FCE7008327C101E3
:102A700003A7C70297E70100938747BE23A0E7009B
:102A80008327C10103A7C702930707009397270075
:102A9000B387E7009397270017E70100130747AEB6
:102AA0003387E7008327C101938747009385070099
:102AB00013050700EFD09FD98327C10103A7C702E1
:102AC00097E701009387079F83A7070083A7C702A3
:102AD0006364F700EFD0DFABEF10103C1300000091
:102AE0008320C1021301010367800000130101FD6F
:102AF000232611022326A100232E01008327C100D3
:102B0000232CF1008327C100639607007370043003
:102B10006F000000EFD01FBF93070500232AF100CC
:102B200003258101EFF09FE31307050093071000D1
:102B30006314F70C97E70100938707B483A7070096
:102B40006390070A8327810103A7C70297E7010063
:102B50009387479683A7070083A7C7026366F7009A
:102B600093071000232EF1008327810193874700EC
:102B700013850700EFD0DFE18327810103A7C70298
:102B800097E70100938787AD83A7070063FCE70001
:102B90008327810103A7C70297E70100938707AC4A
:102BA00023A0E7008327810103A7C702930707003B
:102BB00093972700B387E7009397270017E7010053
:102BC0001307079C3387E70083278101938747001A
:102BD0009385070013050700EFD05FC76F00C001A2
:102BE00083278101938787019385070017E50100FB
:102BF000130545A2EFD09FC5832741011385070028
:102C0000EFD09FAE8327C101138507008320C10247
:102C10001301010367800000130101FE232E110040
:102C2000930800001308000093070000130700003A
:102C3000930600001306004097D501009385853C5C
:102C400017150000130505FBEFF08FAF2326A10039
:102C50000327C100930710006316F700EF20C03A66
:102C60002326A1000327C10093071000631EF7026B
:102C70007370043097E701009387C79F1307F0FF35
:102C800023A0E70097E701009387879D13071000B3
:102C900023A0E70097E701009387079C23A0070084
:102CA000EFD04FF46F0040018327C1006396070007
:102CB000737004306F000000130000008320C10116
:102CC0001301010267800000130101FF2326110098
:102CD0007370043097E701009387879823A007005B
:102CE000EFD09F82130000008320C1001301010177
:102CF0006780000097E701009387079883A7070084
:102D00001387170097E701009387079723A0E70031
:102D10001300000067800000130101FE232E110044
:102D20002326010097E701009387079583A70700F3
:102D300063960700737004306F000000EF10D0112D
:102D400097E701009387479383A707001387F7FF4F
:102D500097E701009387479223A0E70097E70100D8
:102D60009387879183A707006394071697E701006D
:102D70009387478E83A70700638C07146F00800C2E
:102D800097E701009387078983A7C70083A7C70038
:102D90002324F1008327810093878701138507008F
:102DA000EFD01FBF8327810093874700138507005B
:102DB000EFD01FBE8327810003A7C70297E701005A
:102DC0009387C78983A7070063FCE70083278100F7
:102DD00003A7C70297E701009387478823A0E7006E
:102DE0008327810003A7C702930707009397270053
:102DF000B387E7009397270017D701001307477899
:102E00003387E70083278100938747009385070076
:102E100013050700EFD09FA38327810003A7C702F4
:102E200097D701009387076983A7070083A7C70285
:102E3000636AF70097E70100938707831307100081
:102E400023A0E70097D701009387C77C83A70700DB
:102E5000E39807F297E701009387C78083A70700ED
:102E6000638807046F00C003EF00002B9307050081
:102E7000638A070097D701009387077F1307100025
:102E800023A0E70097D701009387C77D83A707009A
:102E90001387F7FF97D701009387C77C23A0E7002C
:102EA00097D701009387077C83A70700E39E07FA63
:102EB00097D701009387477B03A70700930710006C
:102EC0006318F700930710002326F100EFD04FECB2
:102ED000EF10807C8327C100138507008320C10188
:102EE0001301010267800000130101FE232E11006F
:102EF000EF10807697D701009387077683A70700A6
:102F00002326F100EF1040798327C10013850700C5
:102F10008320C1011301010267800000130101FE3B
:102F2000232E1100EFD00FFE930705002326F1009A
:102F300097D701009387477283A707002324F100E6
:102F40008327C10013850700EFD00FFA8327810084
:102F5000138507008320C10113010102678000006F
:102F600097D701009387076F83A707001385070092
:102F700067800000130101FD232611022326A10012
:102F80002324B1002322C100232E01009307500007
:102F9000232CF100EFF01FD697D701009387876BA2
:102FA00083A7070003278100636CF714832781013F
:102FB0009387F7FF232CF1008327C10193975700D4
:102FC0000327C100B306F700032781019307070019
:102FD00093972700B387E7009397270017D701003F
:102FE0001307075AB387E7001306100093850700FD
:102FF00013850600EF108004130705008327C10125
:10300000B387E700232EF10083278101E39007FABD
:103010008327C101939757000327C1003307F700A7
:1030200097D701009387875E83A7070013062000C8
:103030009385070013050700EF10400013070500F4
:103040008327C101B387E700232EF1008327C10145
:10305000939757000327C1003307F70097D7010064
:103060009387075B83A7070013062000938507005B
:1030700013050700EF00907C130705008327C101AB
:10308000B387E700232EF1008327C10193975700F0
:103090000327C100B307F7001306400097D50100CE
:1030A0009385855813850700EF00507913070500B5
:1030B0008327C101B387E700232EF1008327C101D5
:1030C000939757000327C100B307F700130630009A
:1030D00097D501009385C55613850700EF0010763C
:1030E000130705008327C101B387E700232EF100F2
:1030F00083274100638607008327410023A0070040
:10310000EFF09FC18327C101138507008320C1020F
:103110001301010367800000130101FD2326110242
:10312000232E010097D701009387075583A7070037
:10313000639C072297D701009387075283A7070054
:103140001387170097D701009387075123A0E70043
:1031500097D701009387475083A70700232CF100DE
:1031600083278101639C070697D701009387074A4D
:1031700083A7070083A707006386070073700430E6
:103180006F00000097D701009387474883A7070087
:10319000232AF10097D701009387874703A70700E9
:1031A00097D701009387874623A0E70097D70100B0
:1031B000938707460327410123A0E70097D7010023
:1031C0009387C74A83A707001387170097D7010083
:1031D0009387C74923A0E700EF10001097D701009D
:1031E0009387474983A7070003278101636CF71280
:1031F00097D701009387874183A7070083A707001C
:1032000063960700930710006F008000930700008B
:10321000638C070097D701009387C7451307F0FF1A
:1032200023A0E7006F00001097D701009387073EA7
:1032300083A7070083A7C70083A7C7002328F1003F
:103240008327010183A747002326F100032781017B
:103250008327C100637CF70097D7010093878741DC
:103260000327C10023A0E7006F00C00B83270101E3
:103270009387470013850700EFD08FF18327010163
:1032800083A78702638A0700832701019387870149
:1032900013850700EFD0CFEF8327010103A7C702F3
:1032A00097D701009387873B83A7070063FCE7005C
:1032B0008327010103A7C70297D701009387073A25
:1032C00023A0E7008327010103A7C7029307070094
:1032D00093972700B387E7009397270017D701003C
:1032E0001307072A3387E7008327010193874700E5
:1032F0009385070013050700EFD04FD58327010101
:1033000003A7C70297D701009387C71A83A70700AF
:1033100083A7C702E36EF7EC93071000232EF1009A
:103320006FF01FED97D701009387C71883A7070099
:1033300003A7C70297D60100938686249307070048
:1033400093972700B387E70093972700B387F6008A
:1033500003A707009307100063F6E7029307100026
:10336000232EF1006F00000297D701009387872F6B
:1033700083A707001387170097D701009387872E2D
:1033800023A0E70097D701009387072E83A70700A4
:103390006386070093071000232EF1008327C101E5
:1033A000138507008320C102130101036780000019
:1033B000130101FE232E110097D701009387C72B1D
:1033C00083A70700638C070097D701009387C7295D
:1033D0001307100023A0E7006F00C01897D7010063
:1033E0009387872823A0070097D701009387870C2E
:1033F00083A7070083A707032326F100B7A7A5A586
:103400009387575A2324F1008327C10083A707001D
:10341000032781006310F7048327C10093874700C7
:1034200083A70700032781006316F7028327C100E3
:103430009387870083A7070003278100631CF70099
:103440008327C1009387C70083A707000327810054
:103450006302F70697D701009387C70503A7070004
:1034600097D701009387070583A707009387470332
:103470009385070013050700EF4000196F008003D4
:1034800097D701009387871D83A7070063960700DE
:10349000737004306F00000097D701009387071CFA
:1034A00083A707001387F7FF97D701009387071BB0
:1034B00023A0E70097D701009387471A03A70700C7
:1034C00097D601009386C60B9307070093972700B2
:1034D000B387E70093972700B387F60083A7070019
:1034E000E38007FA97D701009387471703A70700E0
:1034F0009307070093972700B387E7009397270068
:1035000017D701001307C707B387E7002322F1008D
:103510008327410083A7470003A747008327410073
:1035200023A2E7008327410003A747008327410028
:1035300093878700631CF7008327410083A7470018
:1035400003A747008327410023A2E7008327410008
:1035500083A7470003A7C70097D70100938787F584
:1035600023A0E700130000008320C1011301010222
:1035700067800000130101FD232611022326A1000C
:103580002324B1008327C1006396070073700430C1
:103590006F00000097D701009387C7F183A707004A
:1035A00093878701938507000325C100EFD0CFB132
:1035B00097D70100938707F083A7070093874700F9
:1035C00013850700EFD0CFBC032781009307F0FFDE
:1035D0006314F70297D701009387C7ED83A707000D
:1035E000938747009385070017D50100130545050C
:1035F000EFD0CFA56F00400297D701009387C70592
:1036000083A7070003278100B307F700232EF100EB
:103610000325C101EF00900B130000008320C102BD
:103620001301010367800000130101FD232611022D
:103630002326A1002324B1002322C1008327C10037
:1036400063960700737004306F00000097D7010085
:103650009387870283A7070063960700737004307F
:103660006F00000097D701009387C7E483A7070086
:10367000832681003707008033E7E60023ACE700AC
:1036800097D70100938707E383A7070093878701F4
:10369000938507000325C100EFD04F9B97D701000A
:1036A000938747E183A707009387470013850700A7
:1036B000EFD00FAE032741009307F0FF6314F7022A
:1036C00097D70100938707DF83A7070093874700F9
:1036D0009385070017D50100130585F6EFD00F97E6
:1036E0006F00400297D70100938707F783A7070071
:1036F00003274100B307F700232EF1000325C10182
:10370000EF00C07C130000008320C10213010103FD
:1037100067800000130101FD232611022326A1006A
:103720002324B1002322C1008327C1006396070030
:10373000737004306F00000097D70100938787D71C
:1037400083A7070093878701938507000325C1009E
:10375000EFD0CF8F97D701009387C7D583A70700F6
:103760009387470013850700EFD08FA203274100FE
:10377000930710006314F70297D70100938787D34C
:1037800083A70700938747009385070017D501009B
:10379000130505EBEFD08F8B6F00400297D7010028
:1037A000938787EB83A7070003278100B307F70000
:1037B000232EF1000325C101EF004071130000002A
:1037C0008320C1021301010367800000130101FD82
:1037D000232611022326A1008327C10083A7C70047
:1037E00083A7C700232CF10083278101639607007C
:1037F000737004306F000000832781019387870175
:1038000013850700EFD0CF9897D701009387C7E6BD
:1038100083A70700639E07068327810193874700DC
:1038200013850700EFD0CF968327810103A7C70236
:1038300097D70100938787E283A7070063FCE7001F
:103840008327810103A7C70297D70100938707E168
:1038500023A0E7008327810103A7C702930707007E
:1038600093972700B387E7009397270017D70100A6
:10387000130707D13387E700832781019387470028
:103880009385070013050700EFC05FFC6F00C001C0
:1038900083278101938787019385070017D501004E
:1038A000130545D7EFC09FFA8327810103A7C702FD
:1038B00097D70100938707C083A7070083A7C70294
:1038C00063F0E70293071000232EF10097D7010061
:1038D000938787D91307100023A0E7006F008000AB
:1038E000232E01008327C101138507008320C10215
:1038F0001301010367800000130101FD232611025B
:103900002326A1002324B10097D701009387C7D6AF
:1039100083A7070063960700737004306F000000F0
:1039200003278100B70700803367F7008327C100B2
:1039300023A0E7008327C10083A7C700232CF10041
:103940008327810163960700737004306F000000C5
:103950000325C100EFD0CF838327810193874700E0
:1039600013850700EFD0CF828327810103A7C70209
:1039700097D70100938787CE83A7070063FCE700F2
:103980008327810103A7C70297D70100938707CD3B
:1039900023A0E7008327810103A7C702930707003D
:1039A00093972700B387E7009397270017D7010065
:1039B000130707BD3387E7008327810193874700FB
:1039C0009385070013050700EFC05FE88327810197
:1039D00003A7C70297D701009387C7AD83A7070046
:1039E00083A7C70263F0E70293071000232EF100BC
:1039F00097D70100938747C71307100023A0E7005C
:103A00006F008000232E01008327C101138507006A
:103A10008320C1021301010367800000130101FF2D
:103A20002326A1008327C10063960700737004302A
:103A30006F00000097D70100938747C303A70700D3
:103A40008327C10023A0E70097D701009387C7C051
:103A500003A707008327C10023A2E700130000008B
:103A60001301010167800000130101FD23261102EB
:103A70002326A1002324B1008327C10063960700F9
:103A8000737004306F000000832781006396070085
:103A9000737004306F000000EF00103C97D70100F6
:103AA000938787BB83A70700232CF100832781001E
:103AB00003A707009307F0FF6316F700232E01000A
:103AC0006F0000098327C10003A7070097D70100F3
:103AD0009387C7B983A707006300F7028327C10054
:103AE00083A74700032781016368F700930710004D
:103AF000232EF1006F00C0058327C10083A7470074
:103B0000032781013307F7408327810083A707003C
:103B1000637CF7028327810003A707008327C10086
:103B200083A6470083278101B387F6403307F70058
:103B30008327810023A0E7000325C100EFF01FEEDB
:103B4000232E01006F00C00093071000232EF10008
:103B5000EF0090348327C101138507008320C10241
:103B6000130101036780000097D701009387C7AF57
:103B70001307100023A0E700130000006780000077
:103B8000130101FE2326A1008327C100638E0700D5
:103B90008327C100232CF1008327810183A7C70459
:103BA000232EF1006F008000232E01008327C10126
:103BB000138507001301010267800000130101FE55
:103BC0002326A1002324B1008327C100638C0700B2
:103BD0008327C100232EF1008327C1010327810021
:103BE00023A6E70413000000130101026780000010
:103BF000130101FE232E11002326A100EF00002156
:103C000097D701009387C79703A707009307100072
:103C1000E3F6E7FEEFC0DF976FF05FFE130101FCF4
:103C2000232E1102232EA100232CB100232AC10030
:103C30002328D100930707002317F1002326010250
:103C40006F004004032781018327C102B307F700F7
:103C500003C707008326C1018327C102B387F6008B
:103C6000238AE702032781018327C102B307F700F4
:103C700083C70700638007028327C1029387170069
:103C80002326F1020327C1029307F000E3FCE7FAC1
:103C90006F008000130000008327C101A381070487
:103CA000032741019307400063F6E70093074000B4
:103CB000232AF1008327C1010327410123A6E7023C
:103CC0008327C1010327410123A8E7048327C101FA
:103CD00023AA07048327C1019387470013850700A0
:103CE000EFC01FB58327C1019387870113850700A4
:103CF000EFC01FB48327C1010327C10123A8E70038
:103D000013075000832741013307F7408327C10180
:103D100023ACE7008327C1010327C10123A2E702E7
:103D20008327C10123A207048327C10123AC070411
:103D30008327C10123AE0704130000008320C103C1
:103D40001301010467800000130101FE232E1100FE
:103D5000232601006F0080030327C100930707009B
:103D600093972700B387E7009397270017D70100A1
:103D700013070781B387E70013850700EFC0DFA5AE
:103D80008327C100938717002326F1000327C10072
:103D900093074000E3F2E7FC17D501001305858483
:103DA000EFC09FA317D5010013050585EFC0DFA263
:103DB00017D5010013050586EFC01FA217D5010016
:103DC00013058586EFC05FA117D501001305458750
:103DD000EFC09FA097D701009387478317D70100B3
:103DE0001307478023A0E70097D7010093874782F6
:103DF00017D701001307478023A0E7001300000036
:103E00008320C1011301010267800000130101FE3C
:103E1000232E11006F008009EFE0DFED97D701003E
:103E20009387878083A7070093B7170093F7F70F4F
:103E30002326F100EFE05FEE8327C10063980706B9
:103E4000EF00900197C701009387077E83A7C70003
:103E500083A7C7002324F1008327810093874700AD
:103E600013850700EFC0DFB297C701009387877EF5
:103E700083A707001387F7FF97C701009387877D04
:103E800023A0E70097C701009387477B83A707001C
:103E90001387F7FF97C701009387477A23A0E700AE
:103EA000EF00807F03258100EF00C03F97C701002E
:103EB0009387C77883A70700E39007F613000000F5
:103EC0008320C1011301010267800000130101FE7C
:103ED000232E11002326A10097C701009387875D39
:103EE00083A707000327C10023A2E70097C70100AB
:103EF0009387877683A707000327C1006378F702BB
:103F000097C701009387C77003A7070097C70100F1
:103F10009387475A83A70700938747009385070035
:103F200013050700EFC05F9A6F00000597C70100F7
:103F30009387C76D03A7070097C70100938787572B
:103F400083A70700938747009385070013050700A1
:103F5000EFC09F9797C701009387C77183A707009A
:103F60000327C100637AF70097C701009387877022
:103F70000327C10023A0E700130000008320C10134
:103F80001301010267800000130101FD23261102C5
:103F9000930705002324B1002317F1008327810034
:103FA000639E07008357E10093972700138507005E
:103FB000EF20C02E930705006F008000832781004B
:103FC000232CF10083278101638A07021305000671
:103FD000EF20C02C232EA1008327C101638A070094
:103FE0008327C1010327810123A8E7026F00400155
:103FF00003258101EF20404A6F008000232E01003D
:104000008327C101638207028327C10103A7070336
:104010008357E10093972700138607009305500A02
:1040200013050700EF20006A8327C10113850700ED
:104030008320C1021301010367800000130101FC0A
:10404000232E1102232C81022326A1002324B10058
:104050002322C100232601028327810083A70700B2
:104060006388071C832781002324F10283278102B0
:1040700083A7470003A747008327810223A2E70005
:104080008327810203A74700832781029387870044
:10409000631CF7008327810283A7470003A747001B
:1040A0008327810223A2E7008327810283A7470099
:1040B00083A7C7002322F102832781002320F10276
:1040C0008327010283A7470003A747008327010234
:1040D00023A2E7008327010203A7470083270102E9
:1040E00093878700631CF7008327010283A747009B
:1040F00003A747008327010223A2E70083270102C9
:1041000083A7470083A7C700232EF1008327C1029E
:10411000939757000327C100B307F7000327C10196
:1041200023A0E7008327C102939757000327C1000C
:10413000B307F7000327C1011307470323A2E700D2
:104140008327C102939757000327C100B307F700E5
:104150000327C1010327870423A4E7008327C102A3
:10416000939757000327C100B307F70003274100C7
:1041700023A6E7008327C102939757000327C100B6
:10418000B307F7000327C1010327C70223A8E700ED
:1041900003274100930730006314F7028327C1010E
:1041A00083A78702638E07008327C1029397570076
:1041B0000327C100B307F7001307200023A6E70079
:1041C0008327C102939757000327C100B307F70065
:1041D0000327C1010327070523AAE7008327C1029C
:1041E000939757000327C100B307F70023AC0700DC
:1041F0008327C10183A607038327C1029397570032
:104200000327C1003304F70013850600EF00C00345
:1042100093070500231EF4008327C102938717002C
:104220002326F1020327C10183274102E316F7E8A1
:104230008327C102138507008320C1030324810360
:104240001301010467800000130101FE2326A10071
:10425000232E01006F00C0018327C1009387170040
:104260002326F1008327C10193871700232EF10035
:104270008327C10003C707009307500AE30EF7FC2A
:104280008327C10193D72700232EF1008327C10183
:104290009397070193D707011385070013010102C4
:1042A00067800000130101FE232E11002326A100C8
:1042B0008327C10083A7070313850700EF20C01DD4
:1042C0000325C100EF20401D130000008320C10121
:1042D0001301010267800000130101FF97C701006D
:1042E0009387C73283A7070083A707006396070059
:1042F000930710006F00800093070000638C070095
:1043000097C70100938707371307F0FF23A0E70043
:104310006F00000397C701009387472F83A707000B
:1043200083A7C70083A7C7002326F1008327C10006
:1043300003A7470097C701009387C73323A0E7006F
:10434000130000001301010167800000130101FF49
:1043500097C701009387071683A707002326F1005C
:104360008327C10013850700130101016780000046
:10437000130101FF97C701009387872E83A70700CA
:1043800063980700930710002326F1006F00400296
:1043900097C701009387472E83A7070063980700FC
:1043A000930720002326F1006F00800023260100E0
:1043B0008327C100138507001301010167800000F6
:1043C000130101FD232611022326A1008327C1002A
:1043D000232EF1008327C100638A07128327C101BE
:1043E00003A7C70297C701009387C70C83A70700DD
:1043F00083A7C702637CF7108327C10183A78701C6
:1044000063C2070297C701009387C70A83A7070003
:1044100083A7C702130750003307F7408327C10162
:1044200023ACE7008327C10183A647018327C1018D
:1044300003A7C7029307070093972700B387E700F6
:104440009397270017C7010013078713B387E70067
:104450006396F600930710006F008000930700003A
:10446000638A07088327C1019387470013850700E4
:10447000EFC00FD297C701009387C70383A7070038
:1044800003A7C7028327C10123A6E7028327C1012F
:1044900003A7C70297C701009387471C83A707009C
:1044A00063FCE7008327C10103A7C70297C7010088
:1044B0009387C71A23A0E7008327C10103A7C70278
:1044C0009307070093972700B387E7009397270088
:1044D00017C701001307C70A3387E7008327C10105
:1044E000938747009385070013050700EFC00FB6B9
:1044F0006F00C00197C701009387C7FB83A7070020
:1045000003A7C7028327C10123A6E7021300000007
:104510008320C1021301010367800000130101FD24
:10452000232611022326A1008327C100232CF1009A
:10453000232E01008327C1006386071097C701005F
:10454000938747F783A70700032781016306F700D6
:10455000737004306F0000008327810183A7470533
:1045600063960700737004306F0000008327810199
:1045700083A747051387F7FF8327810123AAE70451
:104580008327810103A7C7028327810183A707052A
:10459000630AF70A8327810183A747056394070A03
:1045A000832781019387470013850700EFC04FBE23
:1045B0008327810103A707058327810123A6E7023B
:1045C0008327810183A7C702130750003307F740F1
:1045D0008327810123ACE7008327810103A7C7025A
:1045E00097C701009387870783A7070063FCE7004D
:1045F0008327810103A7C70297C701009387070696
:1046000023A0E7008327810103A7C70293070700C0
:1046100093972700B387E7009397270017C70100F8
:10462000130707F63387E700832781019387470045
:104630009385070013050700EFC04FA193071000F3
:10464000232EF1008327C101138507008320C102B7
:1046500013010103678000007370043097C70100E5
:104660009387070083A707006384070297C70100A9
:10467000938747E483A7070003A74704130717009E
:1046800023A2E70497C701009387C7E283A7070027
:10469000130000006780000097C70100938747FC64
:1046A00083A707006384070497C70100938787E007
:1046B00083A7070083A74704638A070297C70100FF
:1046C000938747DF83A7070003A747041307F7FF74
:1046D00023A2E70497C701009387C7DD83A70700DC
:1046E00083A747046394070073600430130000003D
:1046F00067800000130101FF97C70100938787DBE4
:1047000083A7070083A787012326F10097C701002D
:10471000938747DA83A7070003A7C70297C701005B
:10472000938747D983A70700930650003387E64055
:1047300023ACE7008327C1001385070013010101A3
:104740006780000097C701009387C7D683A707003B
:10475000638E070097C701009387C7D583A707001B
:1047600003A747051307170023AAE70497C701000B
:10477000938747D483A7070013850700678000004D
:10478000130101FD232611022326A1002324B100D9
:10479000EFF09FEC97C701009387C7D183A707006D
:1047A00083A787056396070897C70100938787D07B
:1047B00083A707001307100023AEE70483278100B7
:1047C0006388070697C701009387C7CE83A70700B2
:1047D0009387470013850700EFC08F9B0327810055
:1047E0009307F0FF6314F70297C70100938787CC04
:1047F00083A70700938747009385070017C501002B
:10480000130505E4EFC08F846F00400297C70100D5
:10481000938787E483A7070003278100B307F70086
:10482000232EF1000325C101EFF04FEAEFB05FD670
:10483000EFF09FE6EFF05FE297C70100938787C72D
:1048400083A7070083A78705232CF1008327810115
:10485000638C07028327C100638C070097C70100A0
:10486000938747C583A7070023AC07046F00C001E7
:1048700097C70100938707C483A7070003A787058D
:104880001307F7FF23ACE70497C70100938787C29C
:1048900083A7070023AE0704EFF01FE08327810101
:1048A000138507008320C102130101036780000004
:1048B000130101FD232611022326A1002324B100A8
:1048C0002322C1002320D100EFF01FD997C7010098
:1048D000938747BE83A7070003A7C7059307200058
:1048E0006306F70A97C701009387C7BC83A7070031
:1048F00083A687050327C1001347F7FF33F7E600B8
:1049000023ACE70497C701009387C7BA83A70700C2
:104910001307100023AEE70483270100638807060E
:1049200097C70100938707B983A7070093874700BC
:1049300013850700EFC0CF85032701009307F0FF21
:104940006314F70297C701009387C7B683A70700D0
:10495000938747009385070017C50100130545CECF
:10496000EFB0DFEE6F00400297C701009387C7CE1C
:1049700083A7070003270100B307F700232CF100EA
:1049800003258101EFF08FD4EFB09FC0EFF0DFD0AF
:10499000EFF09FCC83274100638E070097C701008B
:1049A000938747B183A7070003A7870583274100A3
:1049B00023A0E70097C701009387C7AF83A707002D
:1049C00003A7C705930710006316F700232E010005
:1049D0006F00C00297C701009387C7AD83A7070088
:1049E00083A68705032781001347F7FF33F7E60007
:1049F00023ACE70493071000232EF10097C70100B2
:104A0000938747AB83A7070023AE0704EFF0DFC807
:104A10008327C101138507008320C102130101030D
:104A200067800000130101FD232611022326A10047
:104A30002324B1002322C1002320D10093071000BA
:104A4000232EF1008327C1006396070073700430A2
:104A50006F0000008327C100232CF100EFF0DFBFBF
:104A600083270100638A07008327810103A7870545
:104A70008327010023A0E7008327810183A7C705BF
:104A8000232AF100832781011307200023AEE704C6
:104A9000032741009307400063ECE70883274100A8
:104AA0001397270097B7010093874756B307F7007E
:104AB00003A7070097B7010093874755B307F7008F
:104AC000678007008327810103A78705832781006B
:104AD0003367F7008327810123ACE7046F004005AB
:104AE0008327810183A78705138717008327810107
:104AF00023ACE7046F00C0038327810103278100F3
:104B000023ACE7046F00C002032741019307200094
:104B1000630AF700832781010327810023ACE704A0
:104B20006F000001232E01006F00800013000000C1
:104B300003274101930710006316F70A83278101B9
:104B40009387470013850700EFB09FE48327810117
:104B500003A7C70297C70100938747B083A7070041
:104B600063FCE7008327810103A7C70297C7010001
:104B70009387C7AE23A0E7008327810103A7C7025D
:104B80009307070093972700B387E70093972700C1
:104B900017C701001307C79E3387E70083278101EA
:104BA000938747009385070013050700EFB01FCADE
:104BB0008327810183A7870263860700737004300F
:104BC0006F0000008327810103A7C70297C7010078
:104BD0009387478E83A7070083A7C70263F4E70084
:104BE000EFB01F9BEFF05FAB8327C1011385070078
:104BF0008320C1021301010367800000130101FC3F
:104C0000232E1102232EA100232CB100232AC10040
:104C10002328D1002326E100930710002326F10268
:104C20008327C10163960700737004306F00000092
:104C30008327C1012324F102EFB0DFAC9307050005
:104C40002322F10283270101638A0700832781025F
:104C500003A787058327010123A0E700832781029B
:104C600083A7C7052320F1028327810213072000B1
:104C700023AEE704032741019307400063ECE708F4
:104C8000832741011397270097B70100938747397E
:104C9000B307F70003A7070097B7010093874738CA
:104CA000B307F700678007008327810203A7870502
:104CB000832781013367F7008327810223ACE70450
:104CC0006F0040058327810283A78705138717009C
:104CD0008327810223ACE7046F00C003832781028E
:104CE0000327810123ACE7046F00C0020327010200
:104CF00093072000630AF7008327810203278101BD
:104D000023ACE7046F000001232601026F0080003E
:104D10001300000003270102930710006314F70E2D
:104D20008327810283A7870263860700737004309C
:104D30006F00000097C701009387079483A70700BF
:104D4000639E070683278102938747001385070028
:104D5000EFB01FC48327810203A7C70297C70100D2
:104D60009387C78F83A7070063FCE700832781022F
:104D700003A7C70297C701009387478E23A0E700C8
:104D80008327810203A7C702930707009397270091
:104D9000B387E7009397270017B701001307477EF3
:104DA0003387E700832781029387470093850700B5
:104DB00013050700EFB09FA96F00C0018327810290
:104DC000938787019385070017C501001305858424
:104DD000EFB0DFA78327810203A7C70297B70100BF
:104DE0009387476D83A7070083A7C70263FCE7008B
:104DF0008327C100638807008327C10013071000C1
:104E000023A0E7008327410213850700EFB0DF8D61
:104E10008327C102138507008320C1031301010406
:104E200067800000130101FD232611022326A10043
:104E30002324B1008327C1006396070073700430F8
:104E40006F0000008327C100232EF100EFB09F8B7D
:104E500093070500232CF1008327C10183A7C70511
:104E6000232AF1008327C1011307200023AEE704A2
:104E70008327C10183A78705138717008327C101F3
:104E800023ACE70403274101930710006314F70ED6
:104E90008327C10183A787026386070073700430EC
:104EA0006F00000097B701009387077D83A7070075
:104EB000639E07068327C101938747001385070078
:104EC000EFB01FAD8327C10103A7C70297B7010049
:104ED0009387C77883A7070063FCE7008327C10196
:104EE00003A7C70297B701009387477723A0E7007E
:104EF0008327C10103A7C7029307070093972700E1
:104F0000B387E7009397270017B701001307476798
:104F10003387E7008327C101938747009385070004
:104F200013050700EFB09F926F00C0018327C101F6
:104F3000938787019385070017B501001305856DD9
:104F4000EFB0DF908327C10103A7C70297B7010025
:104F50009387475683A7070083A7C70263FCE70030
:104F600083278100638807008327810013071000CF
:104F700023A0E7008327810113850700EFB0CFF658
:104F8000130000008320C1021301010367800000A9
:104F9000130101FD232611022326A1008327C1004E
:104FA000232CF10083278101639A070097B7010042
:104FB0009387475083A707006F00800083278101F4
:104FC000232CF100EFF04FE98327810103A7C705E8
:104FD00093072000631CF7008327810123AE070499
:104FE00093071000232EF1006F008000232E010094
:104FF000EFF08FEA8327C101138507008320C102E8
:105000001301010367800000130101FE232E11002C
:1050100023260100EF00500B97B701009387076923
:1050200083A70700638A07029308000013080000A3
:1050300093070000130720009306000013060040AA
:1050400097B50100938505FF170500001305852E10
:10505000EFC01FEF2326A1008327C100639607003E
:10506000737004306F0000008327C10013850700B0
:105070008320C1011301010267800000130101FCBC
:10508000232E1102232EA100232CB100232AC100BC
:105090002328D1002326E10083278101639607009E
:1050A000232601026F0080061305C002EF10001FC7
:1050B0002326A1028327C102638A0704EF00D000E0
:1050C0008327C1020327C10123A0E7008327C10270
:1050D0000327810123ACE7008327C1020327410195
:1050E00023AEE7008327C1020327010123A0E702C3
:1050F0008327C1020327C10023A2E7028327C1023D
:105100009387470013850700EFB08FF28327810153
:1051100063960700737004306F0000008327C1029C
:10512000138507008320C103130101046780000079
:10513000130101FC232E1102232EA100232CB10008
:10514000232AC1002328D1002326E10023260102BF
:105150008327C10163960700737004306F0000005D
:1051600097B701009387875483A70700638C070ACA
:10517000832781012320F102832741012322F102A9
:105180008327C1012324F1020327810193075000E3
:1051900063C6E706EFF0CF9D1307050093072000D5
:1051A0006318F70297B701009387475083A707005A
:1051B00013070102930600000326C10093050700B0
:1051C00013850700EFB01FD22326A1026F008005D0
:1051D00097B701009387874D83A707001307010244
:1051E00093060000130600009305070013850700CF
:1051F000EFB05FCF2326A1026F00C00297B7010076
:105200009387C74A83A7070013070102930600008C
:10521000032601019305070013850700EFB09FF0F7
:105220002326A1028327C102138507008320C1031F
:105230001301010467800000130101FE2326A10071
:105240008327C100232EF1008327C1006396070046
:10525000737004306F0000008327C10183A707002B
:10526000138507001301010267800000130101FD8F
:10527000232611022326A1002324B10097B70100A1
:105280009387474283A7070083A7C70083A7C70068
:10529000232EF1008327C101938747001385070060
:1052A000EFB00FEF8327C10103A7C70193071000D9
:1052B0006310F7068327C10103A787018327C10075
:1052C000B307F7008326C1000326810093850700FA
:1052D0000325C101EF00802213070500930710008A
:1052E0006318F70213070000930600000326C100AD
:1052F000930500000325C101EFF09FE3232CA100DB
:105300008327810163960700737004306F000000EB
:105310008327C10183A747020325C101E780070056
:10532000130000008320C102130101036780000005
:10533000130101FD232611022326A10093078101F9
:1053400013850700EF00800E232EA1008327810123
:10535000938507000325C101EF00C000EF0000287E
:105360006FF0DFFD130101FD232611022326A100AA
:105370002324B100EFD01F98930781011385070004
:10538000EF004011232EA1008327810163960708B7
:1053900083278100639207020327C1008327C1018D
:1053A00063ECE700EFD05F978325C1010325C100BF
:1053B000EFF0DFEB6F008006832781006380070238
:1053C00097B701009387472E83A7070083A707009D
:1053D00093B7170093F7F70F2324F10097B7010055
:1053E0009387C72C83A607000327C1008327C10129
:1053F000B307F74003268100938507001385060055
:10540000EFC01FABEFD05F919307050063980700D3
:10541000EFB00F986F008000EFD01F9013000000D6
:105420008320C1021301010367800000130101FE04
:105430002326A10097B701009387C72683A70700FB
:1054400083A7070093B7170093F7F70F1387070099
:105450008327C10023A0E7008327C10083A707009B
:105460006390070297B701009387C72383A70700BC
:1054700083A7C70083A70700232EF1006F008000D9
:10548000232E01008327C1011385070013010102A8
:1054900067800000130101FD232611022326A100CD
:1054A000EFD09FA4232EA10097B701009387472038
:1054B00083A707000327C101637CF700EF00C02B1F
:1054C0008327C1001307100023A0E7006F00C0006E
:1054D0008327C10023A0070097B701009387471DCA
:1054E0000327C10123A0E7008327C101138507001B
:1054F0008320C1021301010367800000130101FD35
:10550000232611022326A1002324B1002322C10057
:105510002320D100232E01008327C100032781000F
:1055200023A2E7008327C1000327C10023A8E700C7
:10553000032781008327410063E6E7040327410036
:10554000832701003307F7408327C10083A7870122
:105550006368F70093071000232EF1006F00C00668
:1055600097B701009387471403A707008327C1005B
:10557000938747009385070013050700EFB0CFB46A
:105580006F0080040327410083270100637EF7003A
:1055900003278100832701006368F7009307100049
:1055A000232EF1006F00400297B701009387870F09
:1055B00003A707008327C10093874700938507004F
:1055C00013050700EFB04FB08327C1011385070013
:1055D0008320C1021301010367800000130101FD54
:1055E000232611026F0080158327810063C60714EC
:1055F00083270101232EF1008327C10183A74701DF
:10560000638A07008327C10193874700138507003A
:10561000EFB00FB89307410013850700EFF09FE745
:10562000232CA10083278100130790006368F710E3
:105630001397270097B70100938747A0B307F70098
:1056400003A7070097B701009387479FB307F700A9
:10565000678007000327C1008327C10183A7870153
:10566000B307F7000327C100930607000326810153
:10567000938507000325C101EFF05FE813070500DC
:1056800093071000631CF70A8327C10183A7470211
:105690000325C101E78007008327C10103A7C701D4
:1056A00093071000631CF7080327C1008327C1017B
:1056B00083A78701B307F7001307000093060000D4
:1056C00013860700930500000325C101EFF05FA6D4
:1056D000232AA100832741016392070673700430D7
:1056E0006F0000000327C1008327C10123ACE7003E
:1056F0008327C10183A78701639607007370043075
:105700006F0000008327C10103A787018327810160
:10571000B307F700832681010326810193850700E3
:105720000325C101EFF09FDD6F0040010325C1019A
:10573000EF0090566F0080001300000097B7010043
:105740009387C7F683A7070013078100930600001D
:10575000130600009305070013850700EFB05FC52F
:1057600093070500E39207E8130000008320C102BD
:105770001301010367800000130101FD23261102BC
:105780006F00C00E97B701009387C7F183A707008A
:1057900083A7C70083A70700232CF10097B7010058
:1057A000938747F083A7070083A7C70083A7C70095
:1057B000232AF100832741019387470013850700BF
:1057C000EFB00F9D8327410183A7470203254101C5
:1057D000E78007008327410103A7C7019307100053
:1057E0006316F7088327410183A7870103278101F7
:1057F000B307F7002328F100032701018327810164
:1058000063F0E704832741010327010123A2E70096
:10581000832741010327410123A8E70097B701002F
:10582000938747E803A70700832741019387470031
:105830009385070013050700EFB00F896F00000381
:105840001307000093060000032681019305000062
:1058500003254101EFF0DF8D2326A1008327C1003E
:1058600063960700737004306F00000097B7010063
:10587000938747E383A7070083A70700E39407F014
:1058800097B70100938707E283A70700232EF10053
:1058900097B70100938747E103A7070097B7010077
:1058A000938747E023A0E70097B701009387C7DFFE
:1058B0000327C10123A0E700130000008320C102D9
:1058C0001301010367800000130101FF232611006B
:1058D000EFE09FD897B70100938747DD83A70700C4
:1058E0006394070A17B50100130545D9EFA0DFEE51
:1058F00017B501001305C5D9EFA01FEE97B701003A
:10590000938747DA17B70100130747D723A0E700AB
:1059100097B70100938747D917B70100130747D7F7
:1059200023A0E700130600009305C0001305400004
:10593000EFB0CFA21307050097B70100938707D7F1
:1059400023A0E70097B70100938747D683A70700F6
:1059500063960700737004306F00000097B7010072
:105960009387C7D483A707006380070297B7010016
:105970009387C7D383A7070097A501009385856EFA
:1059800013850700EFC0CFC2EFE01FD11300000066
:105990008320C1001301010167800000130101FD94
:1059A000232611022326A1008327C100232EF10004
:1059B0008327C10063960700737004306F000000F6
:1059C000EFE09FC98327C10183A74701B337F000E8
:1059D00093F7F70F232CF100EFE01FCC8327810111
:1059E000138507008320C1021301010367800000B3
:1059F000130101FD232611022326A1008327C100E4
:105A0000232EF1008327C1006396070073700430D2
:105A10006F000000EFE05FC48327C10183A7070286
:105A2000232CF100EFE05FC7832781011385070076
:105A30008320C1021301010367800000130101FDEF
:105A4000232611022326A1002324B1008327C100AD
:105A5000232EF1008327C100639607007370043082
:105A60006F000000EFE05FBF8327C10103278100C3
:105A700023A0E702EFE05FC2130000008320C10211
:105A80001301010367800000130101FE232E1100A2
:105A90001305C001EF0090002326A1008327C10059
:105AA000638E07008327C10023A007008327C1005E
:105AB0009387470013850700EFA01FD28327C100FB
:105AC000138507008320C1011301010267800000D4
:105AD000130101FC232E11022326A1002324B1006F
:105AE0002322C1002320D1008327C1002324F102F7
:105AF0002322010203274100B70700FFB377F70015
:105B000063860700737004306F0000008327410034
:105B100063960700737004306F000000EFE05F854C
:105B2000930705006396070083270100639607002B
:105B3000930710006F008000930700006396070032
:105B4000737004306F000000EFD0CF9A832781027A
:105B500083A707002320F102832581000325C100CC
:105B6000EF00804103270102832781003367F7009C
:105B700083274100B377F70003274100631CF70236
:105B80000327010283278100B367F7002326F10270
:105B90008327810203A707008327410093C7F7FFEC
:105BA0003377F7008327810223A0E7002320010039
:105BB0006F00400483270100638807028327810266
:105BC0009386470003274100B7070005B367F70036
:105BD000032601009385070013850600EFD0DFA49C
:105BE000232601026F0000018327810283A707009B
:105BF0002326F102EFD04F92232EA100832701002C
:105C0000638407088327C10163940700EFA05F98AE
:105C1000EFE05FAE2326A1020327C102B70700020F
:105C2000B377F70063980704EFE01FA3832781028F
:105C300083A707002326F1020327C102832741001F
:105C4000B377F700032741006310F702832781022F
:105C500003A707008327410093C7F7FF3377F700B7
:105C60008327810223A0E700EFE01FA39307100022
:105C70002322F1020327C102B70700019387F7FF30
:105C8000B377F7002326F1028327C10213850700AB
:105C90008320C1031301010467800000130101FB8D
:105CA00023261104232EA100232CB100232AC10096
:105CB0002328D1002326E1008327C101232AF102F2
:105CC000232C0102232801028327C10163960700C8
:105CD000737004306F00000003278101B70700FFD5
:105CE000B377F70063860700737004306F0000001D
:105CF0008327810163960700737004306F000000F2
:105D0000EFE00FE793070500639607008327C100C4
:105D100063960700930710006F0080009307000050
:105D200063960700737004306F000000EFC09FFCA3
:105D30008327410383A707002326F10203260101DD
:105D4000832581010325C102EF00404B2324A102DA
:105D500083278102638C07028327C102232EF1026D
:105D60002326010083274101638807088327410315
:105D700003A707008327810193C7F7FF3377F70055
:105D80008327410323A0E7006F0000078327C1009A
:105D9000639807008327C102232EF1026F00C0051C
:105DA00083274101638A070003278103B7070001A6
:105DB000B367F700232CF10283270101638A0700F0
:105DC00003278103B7070004B367F700232CF10210
:105DD000832741039386470003278101832781039B
:105DE000B367F7000326C1009385070013850600FB
:105DF000EFD09F83232E0102EFC01FF22322A102C6
:105E00008327C10063880708832741026394070042
:105E1000EFA00FF8EFE01F8E232EA1020327C1038E
:105E2000B7070002B377F700639C0704EFE0DF8257
:105E30008327410383A70700232EF10203260101D4
:105E4000832581010325C103EF00403B9307050033
:105E5000638407028327410163800702832741038C
:105E600003A707008327810193C7F7FF3377F70064
:105E70008327410323A0E700EFE01F8223280102CC
:105E80000327C103B70700019387F7FFB377F70034
:105E9000232EF1028327C103138507008320C10449
:105EA0001301010567800000130101FD2326110283
:105EB0002326A1002324B1008327C100232EF10053
:105EC0008327C10063960700737004306F000000E1
:105ED00003278100B70700FFB377F7006386070049
:105EE000737004306F000000EFE00FF78327C101EB
:105EF00083A70700232CF1008327C10103A7070014
:105F00008327810093C7F7FF3377F7008327C10109
:105F100023A0E700EFE04FF88327810113850700F6
:105F20008320C1021301010367800000130101FDFA
:105F3000232611022326A1008327C100232EF1006E
:105F4000EFA04FFC93070500232CF1008327C1012C
:105F500083A70700232AF100832781011385070007
:105F6000EFA08FF883274101138507008320C1022A
:105F70001301010367800000130101FB23261104B4
:105F80002326A1002324B100232C01028327C10072
:105F90002328F102232A01028327C1006396070008
:105FA000737004306F00000003278100B70700FF03
:105FB000B377F70063860700737004306F0000004A
:105FC00083270103938747002326F1028327C10219
:105FD000938787002324F102EFC0DFD18327C1021A
:105FE00083A7C700232EF1028327010303A707001D
:105FF000832781003367F7008327010323A0E7008D
:106000006F00000E8327C10383A747002322F102FC
:106010008327C10383A707002320F102232A01025B
:1060200003270102B70700FFB377F700232EF10023
:1060300003270102B70700019387F7FFB377F70043
:106040002320F1020327C101B7070004B377F7004B
:10605000639207028327010303A707008327010236
:10606000B377F7006388070293071000232AF10231
:106070006F0040028327010303A707008327010263
:10608000B377F700032701026316F70093071000A8
:10609000232AF10283274103638007040327C101F8
:1060A000B7070001B377F700638A0700032781036E
:1060B00083270102B367F700232CF1028327010332
:1060C00003A70700B7070002B367F700938507002F
:1060D0000325C103EFD05F8283274102232EF10203
:1060E0000327C10383278102E31EF7F083270103FF
:1060F00003A707008327810393C7F7FF3377F700D0
:106100008327010323A0E700EFC01FC183270103FA
:1061100083A70700138507008320C104130101052D
:1061200067800000130101FD232611022326A10030
:106130008327C100232EF1008327C10193874700E5
:10614000232CF100EFC01FBB6F00400383278101A8
:1061500003A7C70083278101938787006316F70091
:10616000737004306F0000008327810183A7C7008C
:10617000B705000213850700EFD00FF883278101D0
:1061800083A70700E39407FC0325C101EF00C0309B
:10619000EFC09FB8130000008320C1021301010368
:1061A00067800000130101FE232E11002326A100A9
:1061B0002324B100832581000325C100EFF0DFDB3C
:1061C000130000008320C101130101026780000059
:1061D000130101FE232E11002326A1002324B10068
:1061E000832581000325C100EFF01FCC13000000C0
:1061F0008320C1011301010267800000130101FE29
:106200002326A1002324B1002322C100232E010054
:1062100083274100639007020327C1008327810081
:10622000B377F7006386070293071000232EF1006F
:106230006F0000020327C10083278100B377F700B6
:10624000032781006316F70093071000232EF10047
:106250008327C10113850700130101026780000035
:10626000130101FE2326A1008327C100232CF10086
:106270008327C10063960700232E01006F000001F1
:106280008327810183A78701232EF1008327C10182
:10629000138507001301010267800000130101FC50
:1062A000232E11022326A10023220102EFC09FA466
:1062B000973703009387074183A70700639C070074
:1062C000EF00002C973703009387C73F1307100098
:1062D00023A0E7008327C100638A07029307800099
:1062E000138707008327C100B387E7002326F10047
:1062F0008327C10093F73700638A07008327C10013
:1063000093F7C7FF938747002326F1008327C10037
:10631000638207160327C100B79701009387B7FF71
:1063200063EAE714973703009387C7382324F10201
:10633000973703009387073883A707002326F102C6
:106340006F0080018327C1022324F1028327C10249
:1063500083A707002326F1028327C10283A74700F2
:106360000327C10063F8E7008327C10283A7070062
:10637000E39A07FC0327C10297370300938707348A
:10638000630AF70E8327810283A7070013078000A3
:10639000B387E7002322F1028327C10203A7070086
:1063A0008327810223A0E7008327C10203A74700B8
:1063B0008327C100B307F7401307800013171700A6
:1063C0006378F7080327C1028327C100B307F700EA
:1063D000232EF1008327C10203A747008327C100B2
:1063E0003307F7408327C10123A2E7008327C102B7
:1063F0000327C10023A2E7008327C10183A7470029
:10640000232CF100973703009387C72A2320F1023A
:106410006F0000018327010283A707002320F102F8
:106420008327010283A7070083A747000327810171
:10643000E3E2E7FE8327010203A707008327C101E8
:1064400023A0E700832701020327C10123A0E7005F
:1064500097A701009387470703A707008327C10277
:1064600083A747003307F74097A701009387C70525
:1064700023A0E700EFC05F8A8327410263940700EF
:10648000EF10801783274102138507008320C10383
:106490001301010467800000130101FD232611028E
:1064A0002326A1008327C100232CF1008327C100EC
:1064B0006382070A93078000B307F0400327810136
:1064C000B307F700232CF10083278101232AF10071
:1064D000EFC05F828327410183A747002328F10093
:1064E000973703009387071D232EF1006F000001EB
:1064F0008327C10183A70700232EF1008327C10151
:1065000083A7070083A7470003270101E3E2E7FE13
:106510008327C10103A707008327410123A0E700C8
:106520008327C1010327410123A0E70083274101FD
:1065300003A7470097A70100938707F983A70700E0
:106540003307F70097A70100938707F823A0E70018
:10655000EFC08FFC130000008320C1021301010370
:106560006780000097A70100938707F683A70700BD
:10657000138507006780000013000000678000009B
:10658000130101FF97A701009387071393F7C7FF34
:106590002326F100973703009387C7110327C10013
:1065A00023A0E700973703009387C71023A20700B3
:1065B0009737030093878710379701001307C7FFAA
:1065C00023A2E700973703009387470F23A0070014
:1065D0008327C1002324F10083278100379701001E
:1065E0001307C7FF23A2E7008327810017370300A3
:1065F0001307C70C23A0E7001300000013010101DB
:1066000067800000130101FE2326A1002324B100AE
:106610002322C10083278100232EF1008327C1009C
:10662000232CF1000327C10083278100B367F70003
:1066300093F73700639607066F00C0028327C101F6
:1066400003A707008327810123A0E7008327810197
:1066500093874700232CF1008327C10193874700CC
:10666000232EF100832741009387D7FF0327C10022
:10667000B307F70003278101E362F7FC6F004002D4
:106680000327C10193071700232EF10083278101FF
:1066900093861700232CD100034707002380E700CF
:1066A0000327C10083274100B307F70003278101B7
:1066B000E368F7FC8327C10013850700130101027B
:1066C00067800000130101FE2326A1002324B100EE
:1066D0002322C1000327C10083274100B367F700CD
:1066E00093F73700639807068327810093F7F70F26
:1066F000232AF10083274101939787000327410153
:10670000B367F700232AF10083274101939707011C
:1067100003274101B367F700232AF1008327C10053
:10672000232EF1006F0080018327C10113874700EA
:10673000232EE1000327410123A0E7000327C10026
:1067400083274100B307F7000327C101E36EF7FC7D
:106750006F00C0038327C100232CF1006F00C0012C
:106760008327810113871700232CE1000327810071
:106770001377F70F2380E7000327C1008327410029
:10678000B307F70003278101E36CF7FC8327C100FF
:10679000138507001301010267800000130101FE49
:1067A0002326A1008327C100232EF1006F000001E2
:1067B0008327C10193871700232EF1008327C1018E
:1067C00083C70700E39607FE0327C1018327C100A3
:1067D000B307F7401385070013010102678000002B
:1067E000130101FE2326A1002324B1008327C10049
:1067F000138717002326E10083C70700A30FF100CA
:1068000083278100138717002324E10083C7070033
:10681000230FF1008347F101638807000347F1016B
:106820008347E101E304F7FC0347F1018347E101FA
:10683000B307F740138507001301010267800000CA
:10684000130101FE2326A1002324B1008327C100E8
:10685000232EF10013000000032781009307170087
:106860002324F1008327C10193861700232ED10032
:10687000034707002380E70083C70700E39E07FC68
:106880008327C10013850700130101026780000000
:10689000130101FE2326A100232E0100232C010059
:1068A0006F0000018327C100938717002326F100A2
:1068B0008327C10003C7070093070002E304F7FE24
:1068C0008327C10003C707009307D002630AF700BC
:1068D0008327C10003C707009307B0026312F706BE
:1068E0008327C10083C70700938737FD93B717003D
:1068F00093F7F70F232CF1008327C100938717002C
:106900002326F1006F00C0030327C101930707008E
:1069100093972700B387E70093971700232EF10082
:106920008327C100138717002326E10083C70700D0
:10693000938707FD0327C101B307F700232EF1005A
:106940008327C10083C70700E39007FC83278101E9
:10695000638807008327C101B307F0406F00800000
:106960008327C1011385070013010102678000001E
:10697000130101FE2326A10097370300938787D8D0
:1069800083A707009386170017370300130787D7DD
:106990002320D7000327C1001377F70F9736030092
:1069A000938646DAB387F6002380E7000327C10009
:1069B0009307A000630CF70097370300938787D4F1
:1069C00003A7070093070004631EF704973703002B
:1069D000938747D7232EF1006F00C0038327C1019F
:1069E00013871700232EE10003C70700B70710F035
:1069F000938707F023A0E70097370300938787D09A
:106A000083A707001387F7FF97370300938787CF84
:106A100023A0E700973703009387C7CE83A707001B
:106A2000E39E07FA93070000138507001301010294
:106A300067800000130101EB232611142324811425
:106A40002322911423202115232E3113232C4113AB
:106A5000232A5113232EA100232CB1002328C10087
:106A6000232AD1002326E1002324F100232201015F
:106A7000232601128327C100138A0700930A00000E
:106A8000832701010328410113060A0093860A00A7
:106A90001385070093050800EF10D0419307050008
:106AA0001388050013860700930608008327C11288
:106AB000138717002326E112130706009397270078
:106AC00093060113B387F60023AEE7EE8327C100D8
:106AD00013840700930400008327410113870400F7
:106AE00063E8E70483274101138704006398E70004
:106AF000832701011307040063ECE7028327C10029
:106B00001389070093090000130609009386090002
:106B10000325010183254101EF10005C9307050067
:106B2000138805002328F100232A01016FF09FF448
:106B3000130000006F0040018327C10183258101FC
:106B400003254100E7800700832781001387F7FFB3
:106B50002324E1000327C112E340F7FE6F00400544
:106B60008327C1129397270013070113B307F70078
:106B700003A7C7EF8327C11293972700930601133A
:106B8000B387F60083A6C7EF9307900063F6D7009C
:106B9000930770056F00800093070003B387E70039
:106BA0000327C1018325810113850700E700070042
:106BB0008327C1121387F7FF2326E112E342F0FA7D
:106BC000130000008320C114032481148324411482
:106BD000032901148329C113032A8113832A411332
:106BE0001301011567800000130101FF2326A10096
:106BF0002324B10083268100130710006356D702B7
:106C00008327C10083A707009387770093F787FF47
:106C1000938687000327C1002320D70003A84700DD
:106C200083A707006F0000050327810063040702A4
:106C30000327C10003270700130647008326C1006E
:106C400023A0C600032707009307070013080000CE
:106C50006F0040020327C100032707001306470007
:106C60008326C10023A0C60003270700930707005F
:106C700013080000138507009305080013010101A4
:106C800067800000130101FF2326A1002324B10027
:106C900083268100130710006356D7028327C100A3
:106CA00083A707009387770093F787FF9386870072
:106CB0000327C1002320D70003A8470083A70700AC
:106CC0006F00800503278100630607020327C100C8
:106CD00003270700130647008326C10023A0C60030
:106CE00003270700930707001357F741130807000E
:106CF0006F0080020327C100032707001306470027
:106D00008326C10023A0C6000327070093070700BE
:106D10001357F74113080700138507009305080070
:106D20001301010167800000130101FC232E1102F1
:106D3000232C8102232A91022326A1002324B100BF
:106D40002322C1002320D1006F0040026300043CD5
:106D500083274100938717002322F1008327C10076
:106D60008325810013050400E78007008327410085
:106D700083C707001384070093075002E318F4FC4D
:106D800083274100938717002322F10083274100C6
:106D90002328F10093070002A30BF1009307F0FFF3
:106DA000232EF1009307F0FF232CF1002320010292
:106DB00083274100138717002322E10083C70700C0
:106DC000138407009307D4FD130750056360F7325F
:106DD00013972700979701009387C729B307F700F8
:106DE00003A70700979701009387C728B307F70009
:106DF000678007009307D002A30BF1006FF05FFBE1
:106E000093070003A30BF1006FF09FFA232C0100FE
:106E1000032781019307070093972700B387E700B3
:106E200093971700B307F400938707FD232CF10015
:106E30008327410083C70700138407009307F002EC
:106E400063D287049307900363CE870283274100B0
:106E5000938717002322F1006FF09FFB8327010027
:106E6000138747002320E10083A70700232CF100AC
:106E70006F0080018327C101E3DC07F2232E0100AC
:106E80006FF01FF3130000008327C101E3D207F264
:106E900083278101232EF1009307F0FF232CF100BB
:106EA0006FF01FF183270102938717002320F1025F
:106EB0006FF01FF083270100138747002320E100B4
:106EC00083A707000327C1008325810013850700DE
:106ED000E70007006F004023832701001387470066
:106EE0002320E10083A40700639604009794010027
:106EF0009384C4178327C1016350F00803477101CD
:106F00009307D002630AF706832781019385070060
:106F100013850400EF10001A130705008327C10131
:106F2000B387E740232EF1006F00400283477101D1
:106F30000327C1008325810013850700E7000700B0
:106F40008327C1019387F7FF232EF1008327C10117
:106F5000E34EF0FC6F0040028327C10083258100CF
:106F600013050400E7800700938414008327C10100
:106F70009387F7FF232EF10083C7040013840700D3
:106F80006300040483278101E3C807FC8327810190
:106F90009387F7FF232CF10083278101E3DE07FAB3
:106FA0006F0000028327C1008325810013050002C2
:106FB000E78007008327C1019387F7FF232EF100A5
:106FC0008327C101E340F0FE6F0000149307010026
:106FD0008325010213850700EFF0DFCA9307050040
:106FE000138805002324F10223260103832781024D
:106FF0000328C1029307080063D607048327C10052
:10700000832581001305D002E780070083258102D4
:107010000326C1029307000013080000B386B7409F
:107020001385060033B5A7003307C840B307A74050
:107030001387070093870600130807002324F10233
:10704000232601039307A0002322F1026F004006CC
:107050009307A0002322F1026F0000049307800031
:107060002322F1026F004003930710002320F10256
:107070008327C1008325810013050003E7800700F3
:107080008327C1008325810013058007E78007005F
:10709000930700012322F1029307010083250102D7
:1070A00013850700EFF05FB42324A1022326B10269
:1070B0000327410283477101138807008327C10119
:1070C000032681028326C102832581000325C10096
:1070D000EFF05F966F0040038327C1008325810096
:1070E00013050400E78007006F0000028327C1003A
:1070F0008325810013055002E780070083270101E3
:107100002322F100130000006FF05FC6130000009F
:107110008320C10303248103832441031301010459
:1071200067800000130101FF2326A100B70710F0BC
:10713000938707F20327C10023A0E7006F00000038
:10714000130101FB232611022326A100232AB102E9
:10715000232CC102232ED1022320E1042322F10497
:10716000232401052326110593070105938747FE74
:10717000232EF1008327C101938607000326C10057
:107180009305000017F5FFFF1305C57EEFF0DFB98B
:1071900093070000138507008320C1021301010536
:1071A00067800000130101FE2326A1002324B10003
:1071B0002322710083278100232EF1008327C10140
:1071C00083A707000327C1001377F70F2380E70089
:1071D0008327C10183A70700138717008327C101F5
:1071E00023A0E700130000001301010267800000E4
:1071F000130101FA232E11022326A1002324B1003A
:107200002324C1042326D1042328E104232AF104E2
:10721000232C0105232E1105930701062322F102D9
:107220009307410193054101170600001306C6F7B5
:1072300037F7FFFF9346F7FF37150000130505806A
:107240003388A5003378E8001368783B23A0070152
:107250003305A6003377E5001367773323A2E700F1
:1072600033F7D500931547013787030013073739E4
:1072700033E7E50023A4E7003377D60093164701F0
:10728000370703001307770633E7E60023A6E70076
:107290000F1000008327C1002326F1029307010687
:1072A000938787FE2324F10203278102930741017C
:1072B000138507009307C10093060700032681008A
:1072C00093850700EFF05FA68327C10023800700A6
:1072D0008327C100138707008327C102B307F74044
:1072E000138507008320C103130101066780000096
:1072F000130101FF370510F0130545F403250500C0
:107300002326A100370510F0130505F40325050019
:107310002324A100370510F0130545F403250500CB
:107320008328C100E398A8FC0325C10013030500CE
:107330009303000013170300930600000325810048
:107340009305050013060000B3E7B6003368C700D5
:10735000370710F0130587F4B7150000938505FA79
:1073600013060000B386B70093880600B3B8F80090
:107370003307C800B387E800138707009387060028
:10738000130807002320F500232205011300000045
:107390001301010167800000130101FF2326110082
:1073A000EFF01FF59307000873A0473013000000AB
:1073B0008320C1001301010167800000130101FE59
:1073C000232E11002326A10017950100130505E0C7
:1073D000EFF01FD7130000008320C1011301010249
:1073E00067800000130101FE232E11002326A10057
:1073F00017950100130505DEEFF09FD41300000080
:107400008320C1011301010267800000130101FD07
:10741000232611022326A100232E01006F00400124
:10742000130000008327C10193871700232EF1006A
:107430000327C101B717000093877738E3D2E7FE2F
:1074400017950100130585D9EFF09FCF6FF0DFFC92
:10745000130101FF2326110013050000EF00001C9B
:10746000130000008320C1001301010167800000A8
:10747000130101FE232E110023260100EF00503BD3
:107480001307050093071000630EF700179501001E
:10749000130545D5EFF0DFCA8327C10093E7270026
:1074A0002326F1008327C100138507008320C10133
:1074B0001301010267800000130101FE232E110059
:1074C00023260100EFF0DFF81707000013078706F7
:1074D0009306000013061000930520031795010082
:1074E0001305C5D1EFD09FB92326A1008327C10082
:1074F00063820702EFB05F9F930705001307000048
:107500009306000013860700930510000325C100B1
:10751000EFD01FC223240100EFB00FF0930700004B
:10752000138507008320C101130101026780000059
:10753000130101FD232611022326A10097970100C4
:10754000938787F783A7070013874706979701005C
:10755000938787F623A0E70097970100938707F6A4
:1075600083A707001387470697970100938707F5BE
:1075700023A0E70097970100938707F403A707006C
:107580009307F07C63DEE704979701009387C7F2C7
:1075900083A7070013870783979701009387C7F195
:1075A00023A0E700EFF0DFEC232EA1008327C10129
:1075B000639E070097970100938747F003A7070092
:1075C000B71700009387F77663D0E7028327C101DE
:1075D00013850700EFF01FB5EFB00FEF6F0000014C
:1075E000130000006F008000130000008320C10220
:1075F0001301010367800000737004306F00000006
:107600001300000067800000130101FF2326A10082
:107610002324B100737004306F000000130101FED9
:10762000232E11002326A100930800001308000058
:10763000930700000327C100972603009386861452
:107640001306004097950100938545BC170500007F
:107650001305C50AEFA0DF8E930800001308000091
:10766000930700000327C100972603009386A61105
:1076700013060040979501009385C5B917050000D2
:107680001305C528EFA0DF8B930800001308000046
:10769000930700000327C100972603009386C60EB8
:1076A0001306004097950100938545B71705000024
:1076B0001305454FEFA0DF88930800001308000072
:1076C000930700000327C100972603009386E60B6B
:1076D00013060040979501009385C5B41705000077
:1076E0001305C570EFA0DF85130000008320C101E2
:1076F0001301010267800000130101FB232611041E
:107700002324810423229104232021052326A10080
:10771000231F010297970100938747B103A84700F1
:1077200083A707002328F100232A01018327C10032
:10773000232CF102979701009387C7AF03A8470056
:1077400083A707002328F102232A0103979701004A
:107750009387C7AE03A8470083A707002324F1023D
:1077600023260103979701009387C7AD03A847001D
:1077700083A707002320F1022322010383270103AB
:1077800003284103832681020327C10213860600D2
:10779000930607001385070093050800EF1080414A
:1077A000930705001388050013850700930508005B
:1077B000832701020328410213860700930608006D
:1077C000EF2040609307050013880500232CF1008B
:1077D000232E0101832781010328C1018326010192
:1077E000032741011386060093060700138507004F
:1077F00093050800EF20104C93070500138805003F
:107800001306000093060000138507009305080087
:10781000EF20804B9307050063D80706832781017B
:107820000328C1011384070037070080B344E80030
:1078300083270101032841011386070093060800EE
:107840001305040093850400EF20D046930705003C
:10785000138805001385070093050800130910001D
:10786000979701009387879E03A6070083A647008A
:10787000EF20C035930705006344F00013090000B2
:107880009377F90F6F000006832781010328C10158
:107890008326010103274101138606009306070092
:1078A0001385070093050800EF20D04093070500DB
:1078B00013880500138507009305080013091000BD
:1078C000979701009387879803A6070083A6470030
:1078D000EF20C02F930705006344F0001309000058
:1078E0009377F90F6386070093071000231FF102B7
:1078F0008317E103E39007E4832781031307100054
:107900002390E7006FF01FE3130101FB232611040E
:107910002324810423229104232021052326A1006E
:10792000231F0102979701009387C79203A847007E
:1079300083A707002328F102232A01039797010058
:107940009387C79103A8470083A707002324F10268
:1079500023260103979701009387C79003A8470048
:1079600083A707002320F1022322010383270103B9
:1079700003284103832681020327C10213860600E0
:10798000930607001385070093050800EF101023E6
:107990009307050013880500138507009305080069
:1079A000832701020328410213860700930608007B
:1079B000EF20404193070500138805002328F100BC
:1079C000232A01018327C100232CF102979701008C
:1079D0009387478803A8470083A707002328F1025D
:1079E000232A0103979701009387478703A847003D
:1079F00083A707002324F1022326010397970100A0
:107A00009387478603A8470083A707002320F10236
:107A100023220103832701030328410383268102D4
:107A20000327C1021386060093060700138507008B
:107A300093050800EF1090189307050013880500C0
:107A400013850700930508008327010203284102DC
:107A50001386070093060800EF20C0369307050041
:107A600013880500232CF100232E010183278101B7
:107A70000328C10183260101032741011386060063
:107A8000930607001385070093050800EF20902256
:107A900093070500138805001306000093060000F5
:107AA0001385070093050800EF20002293070500C7
:107AB00063D80706832781010328C10113840700C7
:107AC00037070080B344E800832701010328410100
:107AD000138607009306080013050400938504002D
:107AE000EF20501D9307050013880500138507003C
:107AF0009305080013091000978701009387077505
:107B000003A6070083A64700EF20400C930705005B
:107B10006344F000130900009377F90F6F0000062B
:107B2000832781010328C101832601010327410125
:107B300013860600930607001385070093050800C7
:107B4000EF205017930705001388050013850700E1
:107B50009305080013091000978701009387076FAA
:107B600003A6070083A64700EF2040069307050001
:107B70006344F000130900009377F90F6386070050
:107B800093071000231FF1028317E103E39007E43A
:107B900083278103130710002390E7006FF01FE392
:107BA000130101FB23261104232481042326A100B1
:107BB0009307A000232AF102231D01028327C1009D
:107BC0002328F10283274103939737001385070089
:107BD000EFE0CFEC2326A1022320010223220102A1
:107BE000232C0100232E0100232E01026F00C00967
:107BF0000325C103EF30C00D8327C10393973700DE
:107C00000327C1023304F7009787010093870766B3
:107C100003A6070083A64700EF00D079930705006D
:107C2000138805002320F400232204010325C10347
:107C3000EF30000A978701009387476303A6070088
:107C400083A64700EF00107793070500138805000F
:107C500013850700930508008327010203284102CA
:107C60001386070093060800EF00D0749307050001
:107C7000138805002320F102232201038327C10377
:107C800093871700232EF1020327C10383274103A3
:107C9000E360F7F6232E01026F0040058327C1033E
:107CA000939737000327C102B307F70003A84700E3
:107CB00083A70700832681010327C10113860600DD
:107CC000930607001385070093050800EF00906EE8
:107CD0009307050013880500232CF100232E0101D2
:107CE0008327C10393871700232EF1020327C103C3
:107CF00083274103E364F7FA832701020328410243
:107D0000832681010327C10113860600930607001D
:107D10001385070093050800EF20C079930705003D
:107D2000138805002328F100232A0101832701017C
:107D30000328410113060000930600001385070085
:107D400093050800EF1050789307050063D00704EF
:107D50008327010103284101130410001787010044
:107D600013074751032607008326470013850700A2
:107D700093050800EF1050759307050063C40700D2
:107D8000130400009377F40F6F00C00383270101F1
:107D90000328410113041000178701001307074B44
:107DA0000326070083264700138507009305080074
:107DB000EF10D061930705006344F0001304000046
:107DC0009377F40F6386070093071000231DF102D9
:107DD0008317A103E39207E0832701031307100031
:107DE0002390E7006FF05FDF130101FB23261104EE
:107DF000232481042326A1009307A000232AF10253
:107E0000231D01028327C1002328F1028327410398
:107E10009397370013850700EFE04FC82326A10290
:107E20002320010223220102232C0100232E010022
:107E3000232E01026F00C0090325C103EF20506902
:107E40008327C103939737000327C1023304F70048
:107E5000978701009387874203A6070083A6470000
:107E6000EF10507693070500138805002320F400D7
:107E7000232204010325C103EF20906597870100A9
:107E80009387C73F03A6070083A64700EF109073B0
:107E90009307050013880500138507009305080064
:107EA0008327010203284102138607009306080076
:107EB000EF00505093070500138805002320F102BE
:107EC000232201038327C10393871700232EF10286
:107ED0000327C10383274103E360F7F6232E010242
:107EE0006F0040058327C103939737000327C10222
:107EF000B307F70003A8470083A707008326810183
:107F00000327C101138606009306070013850700A7
:107F100093050800EF00104A930705001388050039
:107F2000232CF100232E01018327C103938717001F
:107F3000232EF1020327C10383274103E364F7FAE9
:107F40008327010203284102832681010327C101FF
:107F500013860600930607001385070093050800A3
:107F6000EF20405593070500138805002328F100F2
:107F7000232A010183270101032841011306000080
:107F8000930600001385070093050800EF10D053F7
:107F90009307050063D007048327010103284101EB
:107FA00013041000178701001307C72C03260700CE
:107FB000832647001385070093050800EF10D05073
:107FC0009307050063C40700130400009377F40FC0
:107FD0006F00C0038327010103284101130410002F
:107FE000178701001307872603260700832647000B
:107FF0001385070093050800EF10503D9307050017
:108000006344F000130400009377F40F63860700C5
:1080100093071000231DF1028317A103E39207E0E9
:1080200083270103130710002390E7006FF05FDF41
:10803000130101FF930710002326F1002324010000
:108040006F008005171703001307C773832781008C
:1080500093971700B307F70083D70700139707011B
:1080600013570701930710006306F700232601004A
:108070006F00C001171703001307C7708327810023
:1080800093971700B307F700239007008327810019
:10809000938717002324F100032781009307300002
:1080A000E3D2E7FA8327C10013850700130101011A
:1080B00067800000B305B500930705006386B7002D
:1080C00003C70700631607003385A74067800000D9
:1080D000938717006FF09FFE130101FD2322910289
:1080E000232A510123261102232481022320210364
:1080F000232E3101232C4101232861012326710104
:1081000023248101232291012320A101930A050048
:1081100093840500639E0638130406009309050046
:10812000178901001309891D63F8C512B7070100FB
:10813000138B05006378F6101307F00F3337C70071
:1081400013173700B357E6003309F90083460900D7
:108150003387E60093060002B386E640638C060090
:10816000B394D40033D7EA003314D600336B9700AE
:10817000B399DA00935A040193850A0013050B00A2
:10818000EF2090461309050093850A00931B040114
:1081900013050B00EF20D04093DB0B019304050087
:1081A0009305050013850B00EF20D03C131909013E
:1081B00093D70901B367F900138A040063FEA7008F
:1081C000B3878700138AF4FF63E8870063F6A7008C
:1081D000138AE4FFB3878700B384A74093850A001E
:1081E00013850400EF2050401309050093850A0011
:1081F00013850400EF20D03A9399090193040500F8
:10820000930505001319090113850B0093D9090182
:10821000EF205036B36939011386040063FCA900CE
:10822000B30934011386F4FF63E6890063F4A900FF
:108230001386E4FF13140A013364C400130A000018
:108240006F000013B707000113070001E36CF6EE9F
:10825000130780016FF01FEF138A0600631A0600F0
:108260009305000013051000EF2090331304050060
:10827000B7070100637EF4129307F00F63F48700E1
:10828000130A8000B35744013309F900034709007A
:108290009306000233074701B386E6406394061253
:1082A000B3848440130A1000135B040193050B0090
:1082B00013850400EF2050331309050093050B00CC
:1082C00013850400931B0401EF20902D93DB0B0119
:1082D000930405009305050013850B00EF209029FA
:1082E0001319090193D70901B367F900938A0400B0
:1082F00063FEA700B3878700938AF4FF63E88700D3
:1083000063F6A700938AE4FFB3878700B384A7408E
:1083100093050B0013850400EF20102D13090500B1
:1083200093050B0013850400EF2090279399090112
:1083300093040500930505001319090113850B002B
:1083400093D90901EF201023B36939011386040082
:1083500063FCA900B30934011386F4FF63E68900C6
:1083600063F4A9001386E4FF13940A013364C40084
:108370001305040093050A008320C102032481022F
:1083800083244102032901028329C101032A8101B7
:10839000832A4101032B0101832BC100032C81009F
:1083A000832C4100032D01001301010367800000AD
:1083B000B7070001130A0001E366F4EC130A800119
:1083C0006FF05FEC3314D40033DAE400B399DA00D1
:1083D00033D7EA00935A0401B394D40093850A007A
:1083E00013050A00336B9700EF20102013090500D6
:1083F00093850A0013050A00931B0401EF20501A0D
:1084000093DB0B01930405009305050013850B0016
:10841000EF2050161319090113570B013367E900B8
:10842000138A0400637EA70033078700138AF4FFD2
:10843000636887006376A700138AE4FF3307870029
:10844000B304A74093850A0013850400EF20D019D8
:108450001309050093850A0013850400EF205014CA
:10846000930405009305050013850B00EF20901081
:1084700013170B011357070113190901B367E9001B
:108480001387040063FEA700B38787001387F4FFF8
:1084900063E8870063F6A7001387E4FFB3878700CC
:1084A000131A0A01B384A740336AEA006FF0DFDFD2
:1084B00063ECD51EB707010063F4F6041307F00F51
:1084C000B335D7009395350033D7B60097870100B1
:1084D0009387C7E2B387E70003C70700130A0002C8
:1084E0003307B700330AEA4063160A021304100088
:1084F000E3E096E833B6CA00134416006FF05FE776
:10850000B707000193050001E3E0F6FC9305800145
:108510006FF09FFBB35CE600B3964601B3ECDC0062
:1085200033D4E40093DB0C01B397440133D7EA0062
:1085300093850B0013050400336BF700B319460154
:10854000EF20900A1309050093850B001305040022
:10855000139C0C01EF20D004135C0C019304050064
:108560009305050013050C00EF20D0001319090135
:1085700013570B013367E90013840400637EA700DF
:10858000330797011384F4FF636897016376A700AC
:108590001384E4FF33079701B304A74093850B00CE
:1085A00013850400EF2050041309050093850B0088
:1085B00013850400EF20C07E930405009305050099
:1085C00013050C00EF20007B93170B011319090111
:1085D00093D70701B367F9001386040063FEA70071
:1085E000B38797011386F4FF63E8970163F6A7004A
:1085F0001386E4FFB387970113140401B70B01003E
:108600003364C4001389FBFF337D240133F929014E
:10861000B384A7409305090013050D00EF20807572
:10862000935C040193050900130B050013850C00EE
:10863000EF20407493D90901130C050093850900BC
:1086400013850C00EF2000731309050093850900C2
:1086500013050D00EF2000723305850193570B01C0
:108660003385A700637485013309790193570501A8
:10867000B387270163E6F402E392F4BCB707010075
:108680009387F7FF3375F50013150501337BFB0066
:1086900033964A0133056501130A0000E37AA6CC3C
:1086A0001304F4FF6FF09FB9130A000013040000D5
:1086B0006FF01FCC130101FB2324810423229104BA
:1086C000232E310323229103232611042320210585
:1086D000232C4103232A51032328610323267103FA
:1086E000232481032320A103232EB101930C050031
:1086F000938905001304050093840500639E0626F4
:1087000013090600138A0600978A0100938A0ABF9C
:1087100063F4C514B70701006376F6129307F00FF0
:1087200063F4C700130A8000B3574601B38AFA0006
:1087300003C70A001305000233074701330AE54067
:10874000630C0A00B395490133D7EC003319460195
:10875000B364B70033944C01935A090193850A001E
:1087600013850400EF2040689309050093850A00F3
:10877000131B090113850400EF208062135B0B01BA
:108780009305050013050B00EF20C05E93990901C6
:1087900093570401B3E7F90063FAA700B3872701F1
:1087A00063E6270163F4A700B3872701B384A740DA
:1087B00093850A0013850400EF20006393090500E8
:1087C00093850A0013850400EF20805D13140401D3
:1087D000930505009399090113050B001354040137
:1087E000EF20405933E48900637AA4003304240164
:1087F000636624016374A400330424013304A44099
:1088000033554401930500008320C10403248104EF
:1088100083244104032901048329C103032A81031A
:10882000832A4103032B0103832BC102032C810202
:10883000832C4102032D0102832DC1011301010587
:1088400067800000B7070001130A0001E36EF6EC31
:10885000130A80016FF05FED631A060093050000B4
:1088600013051000EF20C05313090500B7070100DE
:10887000637AF90E9307F00F63F42701130A80005F
:10888000B3574901B38AFA0003C70A00130500026F
:10889000B384294133074701330AE540E30E0AEA6E
:1088A00033194901B3DAE900B395490133D7EC0034
:1088B00093540901336BB70013850A0093850400B4
:1088C000EF2080529309050093850400931B090152
:1088D00013850A00EF20C04C93DB0B0193050500C4
:1088E00013850B00EF2000499399090193570B0161
:1088F000B3E7F90033944C0163FAA700B38727016B
:1089000063E6270163F4A700B3872701B38AA74072
:108910009385040013850A00EF20004D930905009C
:108920009385040013850A00EF2080479305050016
:1089300013850B00EF20004493150B019399090157
:1089400093D50501B3E5B90063FAA500B385250108
:1089500063E6250163F4A500B3852501B384A54032
:108960006FF09FDFB7070001130A0001E36AF9F017
:10897000130A80016FF0DFF0E3E8D5E8B7070100E4
:1089800063FCF604930BF00F33B5DB0013153500D1
:1089900033D7A6009787010093874796B387E700F0
:1089A00083CB070093050002B38BAB00338B75417B
:1089B000631E0B0263E4360163EACC003384CC40CF
:1089C000B386D94033B58C00B384A64013050400A8
:1089D000938504006FF05FE3B70700011305000102
:1089E000E3E8F6FA130580016FF09FFAB39666018B
:1089F000335D7601336DDD0033D47901B3956901C0
:108A000033DC7C0193540D01336CBC00130504006E
:108A100093850400B31A6601EF20003D130A050098
:108A2000938504001305040033996C01931C0D0118
:108A3000EF20003793DC0C011304050093050500BB
:108A400013850C00EF200033131A0A0113570C0191
:108A50003367EA00130A0400637EA7003307A70107
:108A6000130AF4FF6368A7016376A700130AE4FF03
:108A70003307A701B309A7409385040013850900B4
:108A8000EF20803693850400130405001385090048
:108A9000EF200031930505009304050013850C00B9
:108AA000EF20402D93150C011314040193D50501FB
:108AB000B365B4001387040063FEA500B385A50168
:108AC0001387F4FF63E8A50163F6A5001387E4FFAD
:108AD000B385A501131A0A01B70C0100336AEA0035
:108AE0001384FCFFB3778A0033F48A00B384A54073
:108AF00013850700930504002326F100135A0A0189
:108B0000EF204027930905009305040013050A0090
:108B1000EF20402613DC0A01930D050093050C009D
:108B200013050A00EF2000258327C100130A050062
:108B300093050C0013850700EF20C0233305B50112
:108B400013D709013307A7006374B701330A9A01E9
:108B5000B70701009387F7FF935507013377F700B5
:108B600013170701B3F7F900B3854501B307F70001
:108B700063E6B400639EB400637CF900338657411A
:108B8000B3B7C700B385A541B385F5409307060089
:108B9000B307F9403339F900B385B440B3852541B3
:108BA00033947501B3D767013365F400B3D565011C
:108BB0006FF09FC5370810001308F8FF130101FE7E
:108BC000B378B80013D745019357D5012328210165
:108BD0001379F77F139738003378D800B3E7E700AD
:108BE00013D7460113183800232A91001377F77F13
:108BF00093D8F601232E11009356D601232C810021
:108C00002326310193D4F50133E306011315350012
:108C1000131636003308E9406394143B6354001F75
:108C2000631207143367C3006314070C9306F07FC5
:108C300013070800631CD830B3E6A700639806301A
:108C400093070000130500009396870063DE06007B
:108C5000130717009306F07F630CD774B70680FFE5
:108C60009386F6FFB3F7D7009396D70113553500D7
:108C700033E5A6009306F07F93D73700631ED70035
:108C80003365F5009307000063080500B707080087
:108C90001305000093040000B70610009386F6FF4A
:108CA000B3F7D700B70610801377F77F9386F6FFE8
:108CB00013174701B3F7D700B3E7E7003707008082
:108CC0001347F7FF8320C101032481019395F40129
:108CD000B3F7E70033E7B70083244101032901011B
:108CE0008329C1009305070013010102678000007A
:108CF0009305F8FF639C05043306C5003335A600D1
:108D0000B3876700B387A700130710001305060099
:108D10009396870063DC0622130717009306F07F03
:108D2000E300D7F2B70680FF9386F6FFB3F6D700CD
:108D300093551500137515009397F60133E5A500BB
:108D400033E5A70093D716006F0040201307F07F8C
:108D50006314E80233E7A700630007621307F07F9C
:108D60006F00C01E1307F07FE306E9FE370780009F
:108D70003363E3009305080013078003634EB706CF
:108D80001307F0016342B704130700023307B7402B
:108D9000B356B6003318E3003316E6003368D80044
:108DA0003336C0003368C800B355B3003308A80099
:108DB000B385F500B337A800B387F50013050800A5
:108DC000130709006FF0DFF4130700023358B300F4
:108DD000930600006388E50093060004B385B6405F
:108DE000B316B30033E6C6003336C0003368C8009C
:108DF000930500006FF09FFB3368C3003338000118
:108E00006FF01FFF630A080E631E0908B3E6A70090
:108E1000639206029307F07F6318F7003365C3007F
:108E200093070000E30205E2930703001305060021
:108E30006F00C0119306F0FF631CD8003305C50016
:108E4000B38767003336C500B387C7006FF05FECA8
:108E50009306F07F1348F8FFE302D7FC93068003E4
:108E600063C606099306F00163CA0605930500026E
:108E7000B3850541B3580501B396B7003315B50066
:108E8000B3E616013335A00033E5A60033D8070159
:108E90003305C50033086800B337C500B307F800D1
:108EA0006FF01FE79306F07FE30AD7F6B70680005E
:108EB00033080041B3E7D7006FF05FFA9308000270
:108EC000B3D6070193050000630818019305000459
:108ED00033880541B395070133E5A5003335A0007C
:108EE00033E5A600130800006FF09FFA33E5A700F2
:108EF0003335A0006FF01FFF130719009375F77F3C
:108F00009306100063C8B60833E7A7006314090688
:108F100063080744B366C3001307000063880602B2
:108F20003306C5003335A600B3876700B387A700B3
:108F3000939687001305060063DA0600370780FF63
:108F40001307F7FFB3F7E7001307100093767500D8
:108F5000E38C06CE9376F50013064000E386C6CE7A
:108F60009306450033B5A600B387A7001385060016
:108F70006FF09FCD630C073E3368C300E30008DE4B
:108F8000B7074000130500001307F07F93040000AB
:108F90006FF09FCB9306F07FE304D7CA3306C5007A
:108FA00033886700B337A6003308F8001315F801BB
:108FB000135616003365C500935718006FF01FF95C
:108FC000635E000F6312070A3367C300E30007C63E
:108FD0009306F8FF639E06023306C5403335C5008D
:108FE000B3876740B387A740130710001305060037
:108FF00093968700E3DC06F4370480001304F4FF43
:1090000033F4870093090500130907006F00002758
:109010001307F07FE300E8D413078003634AD708FF
:109020001307F001634ED704130700023307D7403C
:10903000B355D6003318E3003316E6003368B800A2
:109040003336C0003368C800B356D3003308054137
:10905000B386D740B3370501B387F6401305080040
:10906000130709006FF0DFF81307F07FE304E9CE80
:10907000370780003363E300930608006FF0DFF9E1
:10908000130700023358D300130400006388E6007E
:1090900013040004B306D4403314D3003366C40071
:1090A0003336C0003368C800930600006FF01FFA23
:1090B0003368C300333800016FF01FFF630A080EE6
:1090C000631E0908B3E6A700639006029307F07FCA
:1090D0006316F7003365C3006308052A930703008E
:1090E000130506006F00C00F9306F0FF631ED80043
:1090F0003305A640B307F3403336A600B387C74015
:10910000938408006FF0DFEE9306F07F1348F8FFBA
:10911000E302D7FC9306800363C606099306F001B9
:1091200063CA060593050002B3850541335E050158
:10913000B396B7003315B500B3E6C6013335A000CA
:1091400033E5A60033D807013305A64033080341B1
:10915000B337A600B307F8406FF09FFA9306F07F8D
:10916000E30AD7F6B706800033080041B3E7D7001B
:109170006FF05FFA130E0002B3D6070193050000EB
:109180006308C8019305000433880541B3950701BE
:1091900033E5A5003335A00033E5A6001308000031
:1091A0006FF09FFA33E5A7003335A0006FF01FFF83
:1091B000130719001377F77F9306100063CAE608B8
:1091C000B3E6A7003367C30063140906639E060075
:1091D0006302071C93070300130506001307000032
:1091E000938408006FF09FD663000704B306C54060
:1091F000B335D500338767403307B74093158700F1
:1092000063DC05003305A640B307F3403336A60000
:10921000B387C7406FF09FFC33E5E600630A050C97
:109220009307070013850600130700006FF01FD295
:10923000639C0600630807169307030013050600E6
:10924000938408006FF09FB1E30A07B06FF05FD31B
:10925000B309C540338467403338350133040441D2
:109260001317840063520708B309A6403304F34080
:10927000B33736013304F44093840800630E0406C8
:1092800013050400EF10903C130785FF9307F001CE
:1092900063CCE70693070002B387E7403314E4008A
:1092A000B3D7F90033E487003395E9006340270B17
:1092B00033072741930717009306F00163CEF604A6
:1092C000130700023307F7403356F500B316E400E6
:1092D0003315E500B3E6C6003335A00033E5A6003C
:1092E000B357F4006FF05FF433E58900E31805F835
:1092F000930700006F00800A13850900EF101035F6
:10930000130505026FF05FF8130485FD339489009F
:10931000130500006FF09FF9130717FE13060002F4
:109320003357E400930600006388C70093060004E7
:10933000B386F640B316D4003365D5003335A000AC
:109340003365A700930700006FF01FEEB70780FF9B
:109350009387F7FF3307E940B377F4006FF01FBF3F
:1093600093070300130506006FF01FEC930703003B
:10937000130506006FF09F9E930700001305000081
:109380001307F07F6FF05F8C930700009384080051
:109390006FF09F8B93070000130500001307000078
:1093A0006FF0DFBE13050000B70740006FF0DFBDB0
:1093B00093070000130500006FF01F8B130101FBE2
:1093C00023248104232C41033704100013DA4501C0
:1093D00023202105232E3103232A51032324810333
:1093E0001304F4FF2326110423229104232861038C
:1093F00023267103232291032320A103232EB101ED
:10940000137AFA7F13090500130C0600938A0600ED
:109410003374B40093D9F50163060A0A9307F07F09
:109420006304FA1013143400B70780003364F400A7
:10943000135BD501336B8B0093143500130A1AC0EC
:10944000930B000013D54A01370910001309F9FFE7
:109450001375F57F3379590193050C0093DAFA01FE
:10946000630205109307F07F6302F516370480004E
:1094700013193900336989001354DC013364240162
:1094800093153C00130515C09307000013972B009C
:109490003367F7001307F7FF9306E00033C959015C
:1094A000330AAA4063E0E61697760100938686DDCC
:1094B000131727003307D700032707003307D70008
:1094C00067000700336BA400630E0B0663000404FF
:1094D00013050400EF109017930755FF1307C00101
:1094E000634CF702130BD001930485FF330BFB4051
:1094F00033149400335B6901336B8B00B314990010
:10950000130AD0C0330AAA406FF09FF3EF10101473
:10951000130505026FF05FFC130485FD331B890002
:10952000930400006FF0DFFD336BA40063040B02B3
:1095300093040500130B0400130AF07F930B300013
:109540006FF05FF093040000130A0000930B10000B
:109550006FF05FEF93040000130AF07F930B20007D
:109560006FF05FEE33648901630E04066300090443
:1095700013050900EF10900D930755FF1307C00165
:10958000634EF7021304D001930585FF3304F440C2
:109590003319B90033548C0033642401B315BC0073
:1095A0001307D0C03305A7406FF01FEE13050C0062
:1095B000EF10D009130505026FF01FFC130485FDA1
:1095C00033148C00930500006FF09FFD3364890114
:1095D00063020402130409001305F07F93073000AF
:1095E0006FF0DFEA930500001305000093071000F9
:1095F0006FF0DFE9930500001305F07F930720006B
:109600006FF0DFE86366640163128B4863E0B4487F
:109610009316FB0113D71400139CF401135B1B007A
:10962000B3E4E6001314840093DC8501B3EC8C00F2
:1096300093DA0C0193970C0193D70701139D8500D2
:1096400013050B0093850A002322F100EF104075EB
:1096500093050500930B050013950C0113550501A7
:10966000EF1040711304050093850A0013050B00E9
:10967000EF1080771315050113D704013365A70098
:1096800093890B00637E8500330595019389FBFF69
:1096900063689501637685009389EBFF3305950137
:1096A0003304854093850A0013050400EF10406FD2
:1096B00093050500930B050013950C011355050147
:1096C000EF10406B130B050093850A00130504008F
:1096D000EF108071939D04011315050193DD0D01B9
:1096E000B3EDAD0013870B0063FE6D01B38D9D01DB
:1096F0001387FBFF63E89D0163F66D011387EBFFA2
:10970000B38D9D0193960901B7040100B3E6E6000D
:10971000B38D6D41138BF4FF33F76601337B6D011D
:109720001305070093050B0013D406012326D1006F
:109730002324E100EF1000642322A10093050B0015
:1097400013050400EF100063935B0D0193090500FE
:1097500093850B0013050400EF10C06103278100FF
:109760001304050013850B0093050700EF108060BC
:1097700003264100330535018326C1001357060136
:109780003307A700637437013304940037050100E1
:109790001305F5FF93540701B379A70093990901C5
:1097A0003376A600B3848400B389C90063E89D00C2
:1097B0001384060063949D0463723C05330CAC0172
:1097C0003337AC0133079701B38DED001384F6FFF7
:1097D00063E6BC016394BC036362AC0363E69D0073
:1097E000639EB401637C3C01330CAC013337AC01A4
:1097F000330797011384E6FFB38DED00B3093C41B5
:10980000B3849D40B3373C01B384F4409305F0FF2B
:1098100063889C1A93850A0013850400EF10405852
:10982000930505002324A10013950C011355050190
:10983000EF1040542322A10093850A0013850400F1
:10984000EF10805A8326810003274100131505017C
:1098500093D7090133E5A700938D0600637EE500E9
:1098600033059501938DF6FF636895016376E500F6
:10987000938DE6FF33059501B304E54093850A0017
:1098800013850400EF10C051930505002322A100A9
:1098900013950C0113550501EF10C04D130C050075
:1098A00093850A0013850400EF1000549399090171
:1098B000032741001315050193D9090133E5A900D8
:1098C00093070700637E8501330595019307F7FF32
:1098D00063689501637685019307E7FF330595017A
:1098E00093940D01B3E4F4009397040193D7070117
:1098F00093050B00B3098541138507002322F1006E
:1099000093DD0401EF10004793050B00930A050057
:1099100013850D00EF100046130C050093850D0014
:1099200013850B00EF10004583274100130B050042
:1099300013850B0093850700EF10C04333058501A5
:1099400093D70A013385A70063768501B707010025
:10995000330BFB00B70601009386F6FF9357050112
:109960003377D50013170701B3FADA00B38767011D
:109970003307570163E8F900938504006390F90405
:109980006300070433853C019385F4FF636495030A
:109990006366F5006314F5026370ED0293161D0013
:1099A00033BDA601B30C9D019385E4FF33059501FA
:1099B000138D06006314F5006304A70193E51500F9
:1099C0001307FA3F6352E01293F7750063800702B2
:1099D00093F7F50093064000638AD700938645000D
:1099E000B3B5B6003304B400938506009317740032
:1099F00063DA0700B70700FF9387F7FF3374F400BB
:109A000013070A409307E07F63C2E71A9317D40154
:109A100093D53500B3E7B70013543400B7061000F0
:109A20009386F6FF3374D400B70610801377F77F60
:109A30009386F6FF131747013374D4001319F90105
:109A40003364E400336724018320C10403248104C8
:109A500083244104032901048329C103032A8103C8
:109A6000832A4103032B0103832BC102032C8102B0
:109A7000832C4102032D0102832DC10113850700B0
:109A8000930507001301010567800000130AFAFF20
:109A9000130C00006FF01FB91389090013040B00A9
:109AA0009385040093870B00130720006380E71061
:109AB000130730006382E70E13071000E392E7F00C
:109AC00013040000930700006F00400913890A0087
:109AD0006FF09FFD37040800930500001309000094
:109AE000930730006FF05FFC93061000B386E640EA
:109AF00093078003E3C6D7FC9307F00163C4D7063E
:109B0000130AEA41B317440133D7D500339A45010C
:109B1000B3E7E700333A4001B3E747013354D400D9
:109B200013F777006300070213F7F700930640006E
:109B3000630AD70013874700B337F7003304F400F4
:109B40009307070013178400634A07061317D4010D
:109B500093D73700B367F70013543400130700009E
:109B60006FF0DFEB930710FEB387E74013070002A7
:109B7000B357F400130500006386E600130AEA43B6
:109B800033154401336AB500333A4001B3E7470166
:109B9000130400006FF0DFF837040800930700009B
:109BA0001307F07F130900006FF05FE71304000054
:109BB000930700001307F07F6FF05FE613040000C7
:109BC00093070000130710006FF05FE513D74501FE
:109BD000B70710009387F7FF13D8460193080500D5
:109BE000930E05001377F77F1305F07F33F3B7006B
:109BF000130F0600B3F7D70093D5F5011378F87F5C
:109C000093D6F601631AA700336E13011305E0FF24
:109C1000630C0E0867800000631AA80033E6C700D3
:109C20001305E0FF630A0608678000006310070859
:109C300033651301133515006316080033E6C700BA
:109C400063000606631A0500638ED5001305100035
:109C50006396050067800000E39E06FE1305F0FF93
:109C600067800000E344E8FE635A07011305F0FF34
:109C7000E38205FE1305100067800000E3E867FC3F
:109C8000631AF300E364DFFD13050000E3E0EEFF79
:109C90006FF05FFCE36CF3FC1305000067800000CD
:109CA000E31C05FE6FF09FFAE30AE8F613050000D7
:109CB000E30608F86FF05FF9E31807F8336513015E
:109CC000133515006FF01FF813D74501B7071000C3
:109CD0009387F7FF13D8460193080500930E0500FC
:109CE0001377F77F1305F07F33F3B700130F0600E8
:109CF000B3F7D70093D5F5011378F87F93D6F60123
:109D0000631AA700336E130113052000630C0E08BD
:109D100067800000631AA80033E6C700130520001F
:109D2000630A0608678000006310070833651301A3
:109D3000133515006316080033E6C70063000606F6
:109D4000631A0500638ED5001305100063960500A5
:109D500067800000E39E06FE1305F0FF67800000A9
:109D6000E344E8FE635A07011305F0FFE38205FEB2
:109D70001305100067800000E3E867FC631AF30036
:109D8000E364DFFD13050000E3E0EEFF6FF05FFC2E
:109D9000E36CF3FC1305000067800000E31C05FE84
:109DA0006FF09FFAE30AE8F613050000E30608F8EF
:109DB0006FF05FF9E31807F83365130113351500E9
:109DC0006FF01FF8130101FA232C810423263105BB
:109DD0003704100093D94501232A910423206105FB
:109DE000232E7103232C81031304F4FF232E11046B
:109DF000232821052324410523225105232A9103E9
:109E00002328A1032326B10393F9F97F93040500C6
:109E1000930B0600138C06003374B40013DBF501BA
:109E20006388090A9307F07F6386F9103709800079
:109E300013143400336424011359D50133698900A4
:109E4000131D3500938919C0930C000013554C0164
:109E5000370A1000130AFAFF1375F57F337A8A0167
:109E600093840B00135CFC01630405109307F07FDF
:109E70006304F51637048000131A3A00336A8A0027
:109E800013D4DB013364440193943B00130515C0E4
:109E90009307000013972C003367F700B389A900DC
:109EA0001307F7FF9306E000B34B8B01938A190069
:109EB00063E0E61697660100938686401317270035
:109EC0003307D700032707003307D70067000700D1
:109ED0003369A400630E090663000404130504003B
:109EE000EF00D076930755FF1307C001634CF702CC
:109EF0001309D001130D85FF3309F9403314A40170
:109F000033D9240133698900339DA4019309D0C05A
:109F1000B389A9406FF05FF3EF005073130505029A
:109F20006FF05FFC130985FD33992401130D0000C8
:109F30006FF0DFFD3369A40063040902130D05000F
:109F4000130904009309F07F930C30006FF01FF0A9
:109F5000130D000093090000930C10006FF01FEF29
:109F6000130D00009309F07F930C20006FF01FEE9B
:109F700033647A01630E040663000A0413050A00C1
:109F8000EF00D06C930755FF1307C001634EF70233
:109F90001304D001930485FF3304F440331A9A006C
:109FA00033D48B0033644401B3949B009307D0C037
:109FB0003385A7406FF0DFED13850B00EF001069CC
:109FC000130505026FF01FFC130485FD33948B000D
:109FD000930400006FF09FFD33647A016302040272
:109FE00013040A001305F07F930730006FF09FEA17
:109FF0009304000013050000930710006FF09FE921
:10A00000930400001305F07F930720006FF09FE892
:10A0100037070100130AF7FF135C0D0193DD0401FC
:10A02000337D4D01B3F4440193050D001385040005
:10A030002328E100EF001054930C050093850400E1
:10A0400013050C00EF0010532326A10093850D008B
:10A0500013050C00EF001052130B050093050D00C3
:10A0600013850D00EF0010518326C10093D70C011A
:10A070003305D5003385A7006376D500032701019A
:10A08000330BEB009356050133754501B3FC4C01CE
:10A0900013150501B3079501935C04013374440162
:10A0A00093050D0013050400232AD1002326F10097
:10A0B000EF00504C2328A1009305040013050C0069
:10A0C000EF00504B130A050093850C0013050C009C
:10A0D000EF00504A130C050093050D0013850C008A
:10A0E000EF00504903270101330545018326410153
:10A0F000935707013385A70063764501B707010031
:10A10000330CFC003706010093570501338C87019F
:10A110009307F6FF337AF5003377F700131A0A0135
:10A12000135D0901330AEA003379F90033874601E8
:10A1300093050900138504002328E100232EC100A4
:10A14000EF00504393850400232CA10013050D005C
:10A15000EF005042232AA10093050D0013850D0046
:10A16000EF005041930405009305090013850D008D
:10A17000EF00504083264101032781013305D500BC
:10A18000935707013385A7006376D5000326C101E5
:10A19000B384C400B70601009387F6FF935D050101
:10A1A000B3849D00B37DF5003377F7009305090074
:10A1B00013050400939D0D01B38DED00232CD100F8
:10A1C000EF00503B93050400232AA10013050D0066
:10A1D000EF00503A93050D001304050013850C00A1
:10A1E000EF005039130D05009305090013850C008D
:10A1F000EF005038032741013305850093570701CD
:10A200003385A7006376850083268101330DDD0049
:10A2100083270101B70601009386F6FF330BFB008D
:10A22000B377D5003377D70093970701B387E7005B
:10A23000333A4B01B387870133844701330BBB01AA
:10A2400033079400B33DBB01B306B70133BC8701AC
:10A2500033344401935705013337970033648C003E
:10A26000B3BDB6013304F400B36DB7013304B401D8
:10A270003304A40193D77601131494003364F400DB
:10A280008327C10093149B00135B7B01B3E4F400AC
:10A29000B334900093979600B3E46401B3E4F40000
:10A2A0009317740063D2071293D7140093F4140029
:10A2B000B3E497009317F401B3E4F40013541400CB
:10A2C0001387FA3F6356E01093F774006380070228
:10A2D00093F7F40093064000638AD7009387440005
:10A2E000B3B4970033049400938407009317740069
:10A2F00063DA0700B70700FF9387F7FF3374F400B2
:10A3000013870A409307E07F63C6E71893DA3400A7
:10A310009314D401B3E4540113543400B70710006C
:10A320009387F7FF3374F4009377F77F3707108034
:10A330001307F7FF939747013374E400939BFB01E6
:10A340003364F400B36774018320C10503248105DD
:10A350001385040003290105832441058329C104D1
:10A36000032A8104832A4104032B0104832BC103A4
:10A37000032C8103832C4103032D0103832DC10290
:10A38000938507001301010667800000930B0B0003
:10A390001304090093040D0093870C001307200099
:10A3A000638AE70E13073000638CE70C1307100075
:10A3B000E398E7F013040000930400006F008008A6
:10A3C000930B0C006FF09FFD938A09006FF05FEF15
:10A3D00093061000B386E64093078003E3CCD7FCD6
:10A3E0009307F00163C4D706938AEA41B317540177
:10A3F00033D7D400B3945401B3E7E700B3349000EB
:10A40000B3E497003354D40093F7740063800702D9
:10A4100093F7F40013074000638AE7009387440032
:10A42000B3B4970033049400938407009317840017
:10A4300063CA07069317D40193D43400B3E497009A
:10A4400013543400130700006FF05FED930710FE04
:10A45000B387E74013060002B357F4001307000068
:10A460006386C600938AEA4333175401B3649700A6
:10A47000B3349000B3E49700130400006FF0DFF8EA
:10A4800037040800930400001307F07F930B0000CB
:10A490006FF0DFE813040000930400001307F07F5F
:10A4A0006FF0DFE7130400009304000013071000AF
:10A4B0006FF0DFE6370810001308F8FF130101FE04
:10A4C000B378B80013D745019357D5013378D80036
:10A4D000232821011379F77F13973800B3E7E700AA
:10A4E00093D8F60113D74601131838009356D601B6
:10A4F000232A910033E30601232E1100232C81002F
:10A50000232631011377F77F9306F07F93D4F5016B
:10A5100013153500131636006316D700B366C30053
:10A520006394060093C818003308E9406394983A8E
:10A530006354001F631207143367C3006314070CCE
:10A540009306F07F13070800631CD830B3E6A7001A
:10A550006398063093070000130500009396870068
:10A5600063DE0600130717009306F07F630CD774B1
:10A57000B70680FF9386F6FFB3F7D7009396D7010F
:10A580001355350033E5A6009306F07F93D73700C7
:10A59000631ED7003365F5009307000063080500CC
:10A5A000B70708001305000093040000B706100069
:10A5B0009386F6FFB3F7D700B70610801377F77FBF
:10A5C0009386F6FF13174701B3F7D700B3E7E70009
:10A5D000370700801347F7FF8320C101032481015F
:10A5E0009395F401B3F7E70033E7B7008324410103
:10A5F000032901018329C10093050700130101020A
:10A60000678000009305F8FF639C05043306C500CE
:10A610003335A600B3876700B387A7001307100080
:10A62000130506009396870063DC062213071700C4
:10A630009306F07FE300D7F2B70680FF9386F6FF1C
:10A64000B3F6D70093551500137515009397F601CF
:10A6500033E5A50033E5A70093D716006F0040202F
:10A660001307F07F6314E80233E7A7006300076273
:10A670001307F07F6F00C01E1307F07FE306E9FEAB
:10A68000370780003363E300930508001307800356
:10A69000634EB7061307F0016342B70413070002C5
:10A6A0003307B740B356B6003318E3003316E6005D
:10A6B0003368D8003336C0003368C800B355B300E0
:10A6C0003308A800B385F500B337A800B387F500B9
:10A6D00013050800130709006FF0DFF413070002E9
:10A6E0003358B300930600006388E5009306000426
:10A6F000B385B640B316B30033E6C6003336C000A8
:10A700003368C800930500006FF09FFB3368C300F7
:10A71000333800016FF01FFF630A080E631E09083B
:10A72000B3E6A700639206029307F07F6318F70071
:10A730003365C30093070000E30205E293070300BB
:10A74000130506006F00C0119306F0FF631CD800CC
:10A750003305C500B38767003336C500B387C7002C
:10A760006FF05FEC9306F07F1348F8FFE302D7FC2D
:10A770009306800363C606099306F00163CA0605C3
:10A7800093050002B3850541B3580501B396B700A0
:10A790003315B500B3E616013335A00033E5A60046
:10A7A00033D807013305C50033086800B337C50047
:10A7B000B307F8006FF01FE79306F07FE30AD7F6C0
:10A7C000B706800033080041B3E7D7006FF05FFAA7
:10A7D00093080002B3D6070193050000630818012F
:10A7E0009305000433880541B395070133E5A500BF
:10A7F0003335A00033E5A600130800006FF09FFA80
:10A8000033E5A7003335A0006FF01FFF13071900D1
:10A810009375F77F9306100063C8B60833E7A70067
:10A820006314090663080744B366C30013070000F6
:10A83000638806023306C5003335A600B387670078
:10A84000B387A700939687001305060063DA060016
:10A85000370780FF1307F7FFB3F7E7001307100070
:10A8600093767500E38C06CE9376F50013064000D0
:10A87000E386C6CE9306450033B5A600B387A7008E
:10A88000138506006FF09FCD630C073E3368C3004D
:10A89000E30008DEB7074000130500001307F07F50
:10A8A000930400006FF09FCB9306F07FE304D7CAB8
:10A8B0003306C50033886700B337A6003308F800B5
:10A8C0001315F801135616003365C5009357180089
:10A8D0006FF01FF9635E000F6312070A3367C3004E
:10A8E000E30007C69306F8FF639E06023306C540E1
:10A8F0003335C500B3876740B387A74013071000FF
:10A900001305060093968700E3DC06F43704800005
:10A910001304F4FF33F487009309050013090700BB
:10A920006F0000271307F07FE300E8D413078003CC
:10A93000634AD7081307F001634ED70413070002D8
:10A940003307D740B355D6003318E3003316E6007B
:10A950003368B8003336C0003368C800B356D3003C
:10A9600033080541B386D740B3370501B387F640B6
:10A9700013050800130709006FF0DFF81307F07FD5
:10A98000E304E9CE370780003363E3009306080051
:10A990006FF0DFF9130700023358D30013040000EF
:10A9A0006388E60013040004B306D4403314D300D4
:10A9B0003366C4003336C0003368C8009306000015
:10A9C0006FF01FFA3368C300333800016FF01FFFC8
:10A9D000630A080E631E0908B3E6A7006390060227
:10A9E0009307F07F6316F7003365C3006308052AF9
:10A9F00093070300130506006F00C00F9306F0FFD6
:10AA0000631ED8003305A640B307F3403336A600D3
:10AA1000B387C740938408006FF0DFEE9306F07FA2
:10AA20001348F8FFE302D7FC9306800363C60609C8
:10AA30009306F00163CA060593050002B38505413C
:10AA4000335E0501B396B7003315B500B3E6C60112
:10AA50003335A00033E5A60033D807013305A640FF
:10AA600033080341B337A600B307F8406FF09FFAED
:10AA70009306F07FE30AD7F6B7068000330800415B
:10AA8000B3E7D7006FF05FFA130E0002B3D60701E9
:10AA9000930500006308C80193050004338805414D
:10AAA000B395070133E5A5003335A00033E5A600D3
:10AAB000130800006FF09FFA33E5A7003335A000BC
:10AAC0006FF01FFF130719001377F77F930610002D
:10AAD00063CAE608B3E6A7003367C3006314090638
:10AAE000639E06006302071C93070300130506001C
:10AAF00013070000938408006FF09FD663000704DB
:10AB0000B306C540B335D500338767403307B74038
:10AB10009315870063DC05003305A640B307F340B7
:10AB20003336A600B387C7406FF09FFC33E5E600DD
:10AB3000630A050C9307070013850600130700003E
:10AB40006FF01FD2639C060063080716930703008B
:10AB500013050600938408006FF09FB1E30A07B065
:10AB60006FF05FD3B309C540338467403338350194
:10AB7000330404411317840063520708B309A64045
:10AB80003304F340B33736013304F44093840800B0
:10AB9000630E040613050400EF00402B130785FF26
:10ABA0009307F00163CCE70693070002B387E74001
:10ABB0003314E400B3D7F90033E487003395E90098
:10ABC0006340270B33072741930717009306F001D3
:10ABD00063CEF604130700023307F7403356F5003F
:10ABE000B316E4003315E500B3E6C6003335A00024
:10ABF00033E5A600B357F4006FF05FF433E5890046
:10AC0000E31805F8930700006F00800A1385090018
:10AC1000EF00C023130505026FF05FF8130485FDF4
:10AC200033948900130500006FF09FF9130717FE96
:10AC3000130600023357E400930600006388C70040
:10AC400093060004B386F640B316D4003365D500EE
:10AC50003335A0003365A700930700006FF01FEEA7
:10AC6000B70780FF9387F7FF3307E940B377F40016
:10AC70006FF01FBF93070300130506006FF01FEC72
:10AC800093070300130506006FF09F9E93070000D3
:10AC9000130500001307F07F6FF05F8C930700002F
:10ACA000938408006FF09F8B93070000130500004A
:10ACB000130700006FF0DFBE13050000B707400068
:10ACC0006FF0DFBD93070000130500006FF01F8BCE
:10ACD000130101FF232611002324810063040508CA
:10ACE00013040500EF0080161307E0419307A0004E
:10ACF0003307A74063C0A7069307B000B387A740F8
:10AD000013055501B357F4003314A40037051000A0
:10AD10001305F5FFB7061080B3F7A7001377F77F89
:10AD20009386F6FF13174701B3F7D700B3E7E700A1
:10AD3000130504008320C10003248100370700802D
:10AD40001347F7FF33F7E7009305070013010101ED
:10AD500067800000130555FFB317A400130400001B
:10AD60006FF0DFFA930700001304000013070000E0
:10AD70006FF0DFF9130605001305000093F61500C8
:10AD8000638406003305C50093D51500131616001D
:10AD9000E39605FE678000006340050663C605066E
:10ADA00013860500930505001305F0FF630C0602EA
:10ADB00093061000637AB6006358C000131616009D
:10ADC00093961600E36AB6FE1305000063E6C5001D
:10ADD000B385C5403365D50093D6160013561600CB
:10ADE000E39606FE6780000093820000EFF05FFBB1
:10ADF00013850500678002003305A04063D8050075
:10AE0000B305B0406FF0DFF9B305B04093820000A6
:10AE1000EFF01FF93305A040678002009382000025
:10AE200063CA0500634C0500EFF09FF7138505002A
:10AE300067800200B305B040E35805FE3305A0402B
:10AE4000EFF01FF63305B04067800200B70701003E
:10AE5000637AF5029307F00FB3B7A7009397370013
:10AE6000130700023307F740B357F50017550100E9
:10AE70001305C548B307F50003C507003305A74010
:10AE8000678000003707000193070001E36AE5FCD3
:08AE9000930780016FF0DFFC65
:02000004800278
:1000000049444C4500000000244BFEFFBC4AFEFF63
:10001000D84AFEFFF04AFEFF004BFEFFF44CFEFF05
:100020008C4CFEFFA84CFEFFC04CFEFFD04CFEFFE8
:10003000546D7220537663001C56FEFF1C56FEFF63
:100040001C56FEFF0457FEFFAC56FEFFF456FEFFA3
:100050001C56FEFF1C56FEFF0457FEFFAC56FEFF6B
:10006000546D725100000000286E756C6C29000000
:10007000406DFEFF7C70FEFF6870FEFF7C70FEFF2F
:100080007C70FEFF7C70FEFF7C70FEFFEC6DFEFF5F
:100090007C70FEFF7C70FEFF846DFEFF046EFEFF31
:1000A0007C70FEFF906DFEFF9C6DFEFF9C6DFEFF61
:1000B0009C6DFEFF9C6DFEFF9C6DFEFF9C6DFEFF28
:1000C0009C6DFEFF9C6DFEFF9C6DFEFF7C70FEFF35
:1000D0007C70FEFF7C70FEFF7C70FEFF7C70FEFF7C
:1000E0007C70FEFF7C70FEFF7C70FEFF7C70FEFF6C
:1000F0007C70FEFF7C70FEFF7C70FEFF7C70FEFF5C
:100100007C70FEFF7C70FEFF7C70FEFF7C70FEFF4B
:100110007C70FEFF7C70FEFF7C70FEFF7C70FEFF3B
:100120007C70FEFF7C70FEFF7C70FEFF7C70FEFF2B
:100130007C70FEFF7C70FEFF7C70FEFF7C70FEFF1B
:100140007C70FEFF7C70FEFF7C70FEFF7C70FEFF0B
:100150007C70FEFF7C70FEFF7C70FEFF7C70FEFFFB
:100160007C70FEFF7C70FEFF7C70FEFF7C70FEFFEB
:10017000446EFEFF5C6FFEFF7C70FEFF7C70FEFF36
:100180007C70FEFF7C70FEFF7C70FEFF7C70FEFFCB
:100190007C70FEFF346EFEFF7C70FEFF7C70FEFF05
:1001A000EC6FFEFFF86FFEFF7C70FEFF7C70FEFFC1
:1001B000686EFEFF7C70FEFFE06FFEFF7C70FEFF4E
:1001C0007C70FEFF2070FEFF6D69616F750A000094
:1001D0006D69616F75320A0068756E6772790A0021
:1001E0004572726F7220696E20666C6F7073207436
:1001F00061736B73200D0A00436865636B54696D0E
:1002000065720000000000004D617468310000005C
:100210004D617468320000004D6174683300000065
:100220004D617468340000006AE67F50274C41C17C
:100230005305A3923ADD5E4082E2C7985B53A24029
:10024000B29DEFA7C6B18CC0FCA9F1D24D62503F60
:10025000AE47E17A145678C0CDCCCCCC8CBCDF4014
:1002600039D6C56D340000C0000000000000164003
:10027000FCA9F1D24D6250BFE5D022DBF93E284007
:100280002C99FEFF4098FEFF4C98FEFF4098FEFF21
:100290001899FEFF4098FEFF4C98FEFF2C99FEFF38
:1002A0002C99FEFF1899FEFF4C98FEFF1898FEFF50
:1002B0001898FEFF1898FEFF5498FEFFE0A0FEFF7E
:1002C000E0A0FEFF04A1FEFFD4A0FEFFD4A0FEFF2D
:1002D000C4A1FEFF04A1FEFFD4A0FEFFC4A1FEFF47
:1002E000D4A0FEFF04A1FEFFD0A0FEFFD0A0FEFF21
:1002F000D0A0FEFFC4A1FEFF00010202030303031E
:1003000004040404040404040505050505050505A5
:100310000505050505050505060606060606060685
:10032000060606060606060606060606060606066D
:100330000606060606060606070707070707070755
:10034000070707070707070707070707070707073D
:10035000070707070707070707070707070707072D
:10036000070707070707070707070707070707071D
:100370000707070707070707080808080808080805
:1003800008080808080808080808080808080808ED
:1003900008080808080808080808080808080808DD
:1003A00008080808080808080808080808080808CD
:1003B00008080808080808080808080808080808BD
:1003C00008080808080808080808080808080808AD
:1003D000080808080808080808080808080808089D
:1003E000080808080808080808080808080808088D
:0803F0000808080808080808C5
:1003F8001000000000000000017A5200017C010199
:100408001B0D02004C00000018000000C47CFEFF19
:10041800DC05000000440E307089039507810188CF
:100428000292049305940696089709980A990B9ADC
:100438000C0370020AC144C844C944D244D344D40A
:1004480044D544D644D744D844D944DA440E004469
:100458000B00000050000000680000005082FEFF02
:100468000005000000440E50748802890393059922
:100478000B810192049406950796089709980A9AA1
:100488000C9B0D0320010AC144C844C944D244D37B
:1004980044D444D544D644D744D844D944DA44DB78
:0804A800440E00440B000000AB
:1004BC00AAAAAAAA08000000FC8F010004000000F0
:040000058000004037
:00000001FF
